 aamG

 Timestamp is 548ff4b5 (Tue Dec 16 17:00:37 2014)

 Preferred load address is 00010000

 Start         Length     Name                   Class
 0001:00000000 0000ab50H .text                   CODE
 0001:0000ab50 00000b50H .text$yc                CODE
 0001:0000b6a0 00000064H .text$yd                CODE
 0002:00000000 00002d6cH .rdata                  DATA
 0002:00002d6c 0000016cH .rdata$r                DATA
 0002:00002ed8 000000dcH .xdata                  DATA
 0002:00002fb4 000000e8H .xdata$x                DATA
 0002:0000309c 00000000H ATL$__a                 DATA
 0002:0000309c 00000000H ATL$__z                 DATA
 0002:0000309c 00000064H .idata$2                DATA
 0002:00003100 00000014H .idata$3                DATA
 0002:00003114 00000248H .idata$4                DATA
 0002:0000335c 00000324H .idata$6                DATA
 0002:00003680 00000000H .edata                  DATA
 0003:00000000 00000248H .idata$5                DATA
 0003:00000248 00000004H .CRT$XCA                DATA
 0003:0000024c 00000004H .CRT$XCAA               DATA
 0003:00000250 00000004H .CRT$XCL                DATA
 0003:00000254 00000160H .CRT$XCU                DATA
 0003:000003b4 00000004H .CRT$XCZ                DATA
 0003:000003b8 00000004H .CRT$XIA                DATA
 0003:000003bc 00000004H .CRT$XIZ                DATA
 0003:000003c0 00000004H .CRT$XPA                DATA
 0003:000003c4 00000004H .CRT$XPZ                DATA
 0003:000003c8 00000004H .CRT$XTA                DATA
 0003:000003cc 00000004H .CRT$XTZ                DATA
 0003:000003d0 000000ecH .data                   DATA
 0003:000004c0 0000142dH .bss                    DATA
 0004:00000000 00000c30H .pdata                  DATA
 0005:00000000 00000058H .rsrc$01                DATA
 0005:00000060 000003a4H .rsrc$02                DATA

  Address         Publics by Value              Rva+Base       Lib:Object

 0000:00000000       ___safe_se_handler_count   00000000     <absolute>
 0000:00000000       ___safe_se_handler_table   00000000     <absolute>
 0001:00000008       ??1CAAMApp@@QAA@XZ         00011008 f i AAM.obj
 0001:00000054       ?GetApp@@YAPAVCAAMApp@@XZ  00011054 f   AAM.obj
 0001:00000060       ?GetMainWnd@@YAPAVCMainFrame@@XZ 00011060 f   AAM.obj
 0001:00000074       ?WaitForCalibrationDone@@YAXXZ 00011074 f   AAM.obj
 0001:000000d0       ??0CAAMApp@@QAA@XZ         000110d0 f   AAM.obj
 0001:00000128       ?ExitInstance@CAAMApp@@UAAHXZ 00011128 f   AAM.obj
 0001:00000150       ?ReadConnProfileName@CAAMApp@@QAAXXZ 00011150 f   AAM.obj
 0001:000001ac       ?ReadModemName@CAAMApp@@QAAXXZ 000111ac f   AAM.obj
 0001:00000210       ?ReadTimeSetting@CAAMApp@@QAAXXZ 00011210 f   AAM.obj
 0001:00000288       ?GetCarrier@CAAMApp@@QAAXXZ 00011288 f   AAM.obj
 0001:000002a8       ?LoadResourceLibrary@CAAMApp@@QAAHXZ 000112a8 f   AAM.obj
 0001:00000374       ?InitInstance@CAAMApp@@UAAHXZ 00011374 f   AAM.obj
 0001:000004e4       WinMain                    000114e4 f   AAM.obj
 0001:00000578       ??0CArbitrator@@QAA@XZ     00011578 f   Arbitrator.obj
 0001:00000684       ?CloseThread@CArbitrator@@QAAXXZ 00011684 f   Arbitrator.obj
 0001:00000698       ?IsSpiderRunning@CArbitrator@@QAAHXZ 00011698 f   Arbitrator.obj
 0001:00000758       ?CheckProc@CArbitrator@@SAXPAX@Z 00011758 f   Arbitrator.obj
 0001:0000076c       ??1CArbitrator@@UAA@XZ     0001176c f   Arbitrator.obj
 0001:000007e0       ?CreateSession@CArbitrator@@QAAKH@Z 000117e0 f   Arbitrator.obj
 0001:0000081c       ?DeleteSession@CArbitrator@@QAAXH@Z 0001181c f   Arbitrator.obj
 0001:00000824       ?SetUpdaterInProgress@CArbitrator@@QAAX_N@Z 00011824 f   Arbitrator.obj
 0001:00000848       ?SetProvisioningInProgress@CArbitrator@@QAAX_N@Z 00011848 f   Arbitrator.obj
 0001:0000086c       ?SetMDNchanged@CArbitrator@@QAAX_N@Z 0001186c f   Arbitrator.obj
 0001:00000890       ?SetActivationInProgress@CArbitrator@@QAAX_N@Z 00011890 f   Arbitrator.obj
 0001:000008b4       ?GetMDNchanged@CArbitrator@@QAA_NXZ 000118b4 f   Arbitrator.obj
 0001:000008d8       ?GetProvisioningStatus@CArbitrator@@QAA_NXZ 000118d8 f   Arbitrator.obj
 0001:000008fc       ?SetCheckPDP@CArbitrator@@QAAX_N@Z 000118fc f   Arbitrator.obj
 0001:00000928       ?IsRunning@CArbitrator@@QAAHPAG@Z 00011928 f   Arbitrator.obj
 0001:00000a48       ??_ECArbitrator@@UAAPAXI@Z 00011a48 f i Arbitrator.obj
 0001:00000a48       ??_GCArbitrator@@UAAPAXI@Z 00011a48 f i Arbitrator.obj
 0001:00000a6c       ?StartThread@CArbitrator@@QAAXXZ 00011a6c f   Arbitrator.obj
 0001:00000ab0       ?RebootDevice@CArbitrator@@QAAXXZ 00011ab0 f   Arbitrator.obj
 0001:00000b6c       ?LaunchIOTA@CArbitrator@@QAAXK@Z 00011b6c f   Arbitrator.obj
 0001:00000d50       ?CheckProcRun@CArbitrator@@UAAXXZ 00011d50 f   Arbitrator.obj
 0001:000011d0       ??0CIota24Dlg@@QAA@XZ      000121d0 f   iota24dlg.obj
 0001:000011e8       ??1CIota24Dlg@@UAA@XZ      000121e8 f   iota24dlg.obj
 0001:000011f8       ??_ECIota24Dlg@@UAAPAXI@Z  000121f8 f i iota24dlg.obj
 0001:000011f8       ??_GCIota24Dlg@@UAAPAXI@Z  000121f8 f i iota24dlg.obj
 0001:00001224       ??0CMainFrame@@QAA@XZ      00012224 f   MainFrm.obj
 0001:000015e4       ??1CMainFrame@@UAA@XZ      000125e4 f   MainFrm.obj
 0001:0000190c       ?OnUSSDNotification@CMainFrame@@QAAJIJ@Z 0001290c f   MainFrm.obj
 0001:00001960       ?OnMIPFailEvent@CMainFrame@@QAAJIJ@Z 00012960 f   MainFrm.obj
 0001:00002020       ?InsertWPSBubble@CMainFrame@@QAAXXZ 00013020 f   MainFrm.obj
 0001:000021d8       ?RemoveWPSBubble@CMainFrame@@QAAXXZ 000131d8 f   MainFrm.obj
 0001:00002268       ?RemoveEmergencyICon@CMainFrame@@QAAXXZ 00013268 f   MainFrm.obj
 0001:000022a8       ?RemovePhoneBubbleICon@CMainFrame@@QAAXXZ 000132a8 f   MainFrm.obj
 0001:000022f0       ?UpdateEmergencyICon@CMainFrame@@QAAXH@Z 000132f0 f   MainFrm.obj
 0001:000024b8       ?InsertEmergencyICon@CMainFrame@@QAAXXZ 000134b8 f   MainFrm.obj
 0001:00002674       ?OnEmergencyHangUp@CMainFrame@@QAAJIJ@Z 00013674 f   MainFrm.obj
 0001:00002720       ?OnSubscriberNumber@CMainFrame@@QAAJIJ@Z 00013720 f   MainFrm.obj
 0001:00002ba4       ?OnDataCallStatusEvent@CMainFrame@@QAAJIJ@Z 00013ba4 f   MainFrm.obj
 0001:00002c58       ?CheckForDataCall@CMainFrame@@QAA_NXZ 00013c58 f   MainFrm.obj
 0001:00002cf4       ?OnResultGetMinActiveState@CMainFrame@@QAAJIJ@Z 00013cf4 f   MainFrm.obj
 0001:00002ff4       ?OnResultCallbackError@CMainFrame@@QAAJIJ@Z 00013ff4 f   MainFrm.obj
 0001:00003038       ?On1XPdpInactFailEvent@CMainFrame@@QAAJIJ@Z 00014038 f   MainFrm.obj
 0001:00003124       ?OnResultGetSystemTime@CMainFrame@@QAAJIJ@Z 00014124 f   MainFrm.obj
 0001:00003164       ?OnPwrStateUpdate@CMainFrame@@QAAJIJ@Z 00014164 f   MainFrm.obj
 0001:000031f8       ?OnSrvStateUpdate@CMainFrame@@QAAJIJ@Z 000141f8 f   MainFrm.obj
 0001:00003284       ?OnSIPNAIPWD@CMainFrame@@QAAJIJ@Z 00014284 f   MainFrm.obj
 0001:00003368       ?WndProc@@YAJPAUHWND__@@IIJ@Z 00014368 f   MainFrm.obj
 0001:0000339c       ?MyRegisterClass@@YAGPAUHINSTANCE__@@PAG@Z 0001439c f   MainFrm.obj
 0001:00003430       ?Create@CMainFrame@@QAAHXZ 00014430 f   MainFrm.obj
 0001:000034fc       ??_ECMainFrame@@UAAPAXI@Z  000144fc f i MainFrm.obj
 0001:000034fc       ??_GCMainFrame@@UAAPAXI@Z  000144fc f i MainFrm.obj
 0001:00003528       ?OnAllCallStatusEvent@CMainFrame@@QAAJIJ@Z 00014528 f   MainFrm.obj
 0001:00003ac0       ?WindowProc@CMainFrame@@UAAJIIJ@Z 00014ac0 f   MainFrm.obj
 0001:0000432c       ??0CMipErrorDlg@@QAA@K@Z   0001532c f   miperrdlg.obj
 0001:00004348       ??1CMipErrorDlg@@UAA@XZ    00015348 f   miperrdlg.obj
 0001:00004358       ?MipErrDlgProc@CMipErrorDlg@@SAHPAUHWND__@@IIJ@Z 00015358 f   miperrdlg.obj
 0001:00004484       ?SetMessageText@CMipErrorDlg@@QAAXI@Z 00015484 f   miperrdlg.obj
 0001:000044f8       ?SetErrId@CMipErrorDlg@@QAAXH@Z 000154f8 f   miperrdlg.obj
 0001:0000456c       ?ShowWindow@CMipErrorDlg@@QAAXH@Z 0001556c f   miperrdlg.obj
 0001:00004584       ?BringWindowToTop@CMipErrorDlg@@QAAHXZ 00015584 f   miperrdlg.obj
 0001:000045a0       ?Initialize@CMipErrorDlg@@QAAXXZ 000155a0 f   miperrdlg.obj
 0001:000046c0       ??_GCMipErrorDlg@@UAAPAXI@Z 000156c0 f i miperrdlg.obj
 0001:000046c0       ??_ECMipErrorDlg@@UAAPAXI@Z 000156c0 f i miperrdlg.obj
 0001:000046e4       ?Create@CMipErrorDlg@@QAAHPAUHWND__@@@Z 000156e4 f   miperrdlg.obj
 0001:000047e8       ??0CResultListElement@@QAA@XZ 000157e8 f   resultelement.obj
 0001:00004800       ??1CResultListElement@@UAA@XZ 00015800 f   resultelement.obj
 0001:00004810       ?SetCallBackId@CResultListElement@@QAAXJ@Z 00015810 f   resultelement.obj
 0001:00004818       ?GetCallBackId@CResultListElement@@QAAJXZ 00015818 f   resultelement.obj
 0001:00004820       ?SetFuncId@CResultListElement@@QAAXW4eFuncId@1@@Z 00015820 f   resultelement.obj
 0001:00004828       ?GetFuncId@CResultListElement@@QAA?AW4eFuncId@1@XZ 00015828 f   resultelement.obj
 0001:00004830       ??_ECResultListElement@@UAAPAXI@Z 00015830 f i resultelement.obj
 0001:00004830       ??_GCResultListElement@@UAAPAXI@Z 00015830 f i resultelement.obj
 0001:00004854       ?GetSessionId@CSession@@QAAHXZ 00015854 f   Session.obj
 0001:00004878       ?AppCheckTimer@@YAXPAUHWND__@@IIK@Z 00015878 f   Session.obj
 0001:0000487c       ?GetSessionName@CSession@@QAAXPAG@Z 0001587c f   Session.obj
 0001:0000488c       ??0CSession@@QAA@XZ        0001588c f   Session.obj
 0001:000048cc       ??_ECSession@@UAAPAXI@Z    000158cc f i Session.obj
 0001:000048cc       ??_GCSession@@UAAPAXI@Z    000158cc f i Session.obj
 0001:00004908       ?Create@CSession@@QAAKH@Z  00015908 f   Session.obj
 0001:00004944       ??1bad_alloc@std@@UAA@XZ   00015944 f i SessionManager.obj
 0001:00004958       ??_Gbad_alloc@std@@UAAPAXI@Z 00015958 f i SessionManager.obj
 0001:00004958       ??_Ebad_alloc@std@@UAAPAXI@Z 00015958 f i SessionManager.obj
 0001:00004988       ??E?$_Const_iterator@$00@?$list@PAVCSession@@V?$allocator@PAVCSession@@@std@@@std@@QAAAAV012@XZ 00015988 f i SessionManager.obj
 0001:000049c4       ??8?$_Const_iterator@$00@?$list@PAVCSession@@V?$allocator@PAVCSession@@@std@@@std@@QBA_NABV012@@Z 000159c4 f i SessionManager.obj
 0001:00004a0c       ?_Inside@?$basic_string@DU?$char_traits@D@std@@V?$allocator@D@2@@std@@IAA_NPBD@Z 00015a0c f i SessionManager.obj
 0001:00004a4c       ??$_Allocate@U_Node@?$_List_nod@PAVCSession@@V?$allocator@PAVCSession@@@std@@@std@@@std@@YAPAU_Node@?$_List_nod@PAVCSession@@V?$allocator@PAVCSession@@@std@@@0@IPAU120@@Z 00015a4c f i SessionManager.obj
 0001:00004abc       ??$_Allocate@D@std@@YAPADIPAD@Z 00015abc f i SessionManager.obj
 0001:00004b28       ??0bad_alloc@std@@QAA@ABV01@@Z 00015b28 f i SessionManager.obj
 0001:00004b48       ?clear@?$list@PAVCSession@@V?$allocator@PAVCSession@@@std@@@std@@QAAXXZ 00015b48 f i SessionManager.obj
 0001:00004b8c       ?erase@?$list@PAVCSession@@V?$allocator@PAVCSession@@@std@@@std@@QAA?AV?$_Iterator@$00@12@V312@@Z 00015b8c f i SessionManager.obj
 0001:00004c14       ?_Tidy@?$basic_string@DU?$char_traits@D@std@@V?$allocator@D@2@@std@@IAAX_NI@Z 00015c14 f i SessionManager.obj
 0001:00004c74       ?_Buynode@?$list@PAVCSession@@V?$allocator@PAVCSession@@@std@@@std@@IAAPAU_Node@?$_List_nod@PAVCSession@@V?$allocator@PAVCSession@@@std@@@2@XZ 00015c74 f i SessionManager.obj
 0001:00004c98       ?erase@?$basic_string@DU?$char_traits@D@std@@V?$allocator@D@2@@std@@QAAAAV12@II@Z 00015c98 f i SessionManager.obj
 0001:00004d2c       ?_Buynode@?$list@PAVCSession@@V?$allocator@PAVCSession@@@std@@@std@@IAAPAU_Node@?$_List_nod@PAVCSession@@V?$allocator@PAVCSession@@@std@@@2@PAU342@0ABQAVCSession@@@Z 00015d2c f i SessionManager.obj
 0001:00004d70       ?_Copy@?$basic_string@DU?$char_traits@D@std@@V?$allocator@D@2@@std@@IAAXII@Z 00015d70 f i SessionManager.obj
 0001:00004ec0       ?DeleteSession@CSessionManager@@QAA_NH@Z 00015ec0 f   SessionManager.obj
 0001:00004fc8       ?IsAppRunning@CSessionManager@@QAA_NH@Z 00015fc8 f   SessionManager.obj
 0001:0000507c       ?Check@CSessionManager@@QAAKH@Z 0001607c f   SessionManager.obj
 0001:00005230       ??1?$basic_string@DU?$char_traits@D@std@@V?$allocator@D@2@@std@@QAA@XZ 00016230 f i SessionManager.obj
 0001:0000523c       ??1?$list@PAVCSession@@V?$allocator@PAVCSession@@@std@@@std@@QAA@XZ 0001623c f i SessionManager.obj
 0001:0000525c       ?_Grow@?$basic_string@DU?$char_traits@D@std@@V?$allocator@D@2@@std@@IAA_NI_N@Z 0001625c f i SessionManager.obj
 0001:00005300       ??1logic_error@std@@UAA@XZ 00016300 f i SessionManager.obj
 0001:0000532c       ?what@logic_error@std@@UBAPBDXZ 0001632c f i SessionManager.obj
 0001:00005344       ??_Elogic_error@std@@UAAPAXI@Z 00016344 f i SessionManager.obj
 0001:00005344       ??_Glogic_error@std@@UAAPAXI@Z 00016344 f i SessionManager.obj
 0001:0000538c       ??1CSessionManager@@UAA@XZ 0001638c f   SessionManager.obj
 0001:0000547c       ?assign@?$basic_string@DU?$char_traits@D@std@@V?$allocator@D@2@@std@@QAAAAV12@ABV12@II@Z 0001647c f i SessionManager.obj
 0001:00005540       ?assign@?$basic_string@DU?$char_traits@D@std@@V?$allocator@D@2@@std@@QAAAAV12@PBDI@Z 00016540 f i SessionManager.obj
 0001:000055e0       ??0CSessionManager@@QAA@XZ 000165e0 f   SessionManager.obj
 0001:00005620       ??_GCSessionManager@@UAAPAXI@Z 00016620 f i SessionManager.obj
 0001:00005620       ??_ECSessionManager@@UAAPAXI@Z 00016620 f i SessionManager.obj
 0001:0000564c       ??0logic_error@std@@QAA@ABV?$basic_string@DU?$char_traits@D@std@@V?$allocator@D@2@@1@@Z 0001664c f i SessionManager.obj
 0001:000056c4       ??1length_error@std@@UAA@XZ 000166c4 f i SessionManager.obj
 0001:000056f0       ??_Elength_error@std@@UAAPAXI@Z 000166f0 f i SessionManager.obj
 0001:000056f0       ??_Glength_error@std@@UAAPAXI@Z 000166f0 f i SessionManager.obj
 0001:00005730       ??0?$basic_string@DU?$char_traits@D@std@@V?$allocator@D@2@@std@@QAA@PBD@Z 00016730 f i SessionManager.obj
 0001:00005770       ?_Incsize@?$list@PAVCSession@@V?$allocator@PAVCSession@@@std@@@std@@IAAXI@Z 00016770 f i SessionManager.obj
 0001:00005820       ??0logic_error@std@@QAA@ABV01@@Z 00016820 f i SessionManager.obj
 0001:00005898       ??0length_error@std@@QAA@ABV01@@Z 00016898 f i SessionManager.obj
 0001:000058c0       ?CreateSession@CSessionManager@@QAAKH@Z 000168c0 f   SessionManager.obj
 0001:000059b8       ??0CStateMachineMgr@@QAA@XZ 000169b8 f   StateMachineMgr.obj
 0001:00005a3c       ?CheckPhoneActivated@CStateMachineMgr@@QAA_NXZ 00016a3c f   StateMachineMgr.obj
 0001:00005a60       ?SetPhoneStatusCheck@CStateMachineMgr@@QAAX_N@Z 00016a60 f   StateMachineMgr.obj
 0001:00005a84       ?GetPhoneStatusCheck@CStateMachineMgr@@QAA_NXZ 00016a84 f   StateMachineMgr.obj
 0001:00005aa8       ?SetDeferredIOTATrigger@CStateMachineMgr@@QAAX_N@Z 00016aa8 f   StateMachineMgr.obj
 0001:00005acc       ?GetDeferredIOTATrigger@CStateMachineMgr@@QAA_NXZ 00016acc f   StateMachineMgr.obj
 0001:00005af0       ?GetServiceStatus@CStateMachineMgr@@QAA?AW4ServiceStatus@@XZ 00016af0 f   StateMachineMgr.obj
 0001:00005b1c       ?HangUpActiveDataCall@CStateMachineMgr@@QAA_NXZ 00016b1c f   StateMachineMgr.obj
 0001:00005c2c       ?SetPhoneActiveState@CStateMachineMgr@@QAAX_N@Z 00016c2c f   StateMachineMgr.obj
 0001:00005c50       ?SetSvcStatus@CStateMachineMgr@@QAAXW4ServiceStatus@@@Z 00016c50 f   StateMachineMgr.obj
 0001:00005c74       ?SetDataCallStatus@CStateMachineMgr@@QAAXW4DataCallStatus@@@Z 00016c74 f   StateMachineMgr.obj
 0001:00005c98       ?GetDataCallStatus@CStateMachineMgr@@QAA?AW4DataCallStatus@@XZ 00016c98 f   StateMachineMgr.obj
 0001:00005cbc       ?SetAALDeferredIOTATrigger@CStateMachineMgr@@QAAX_N@Z 00016cbc f   StateMachineMgr.obj
 0001:00005ce0       ?GetAALDeferredIOTATrigger@CStateMachineMgr@@QAA_NXZ 00016ce0 f   StateMachineMgr.obj
 0001:00005d04       ?SetCallStatus@CStateMachineMgr@@QAAXW4CallStatus@@@Z 00016d04 f   StateMachineMgr.obj
 0001:00005d28       ?GetCallStatus@CStateMachineMgr@@QAA?AW4CallStatus@@XZ 00016d28 f   StateMachineMgr.obj
 0001:00005d4c       ??_GCStateMachineMgr@@UAAPAXI@Z 00016d4c f i StateMachineMgr.obj
 0001:00005d4c       ??_ECStateMachineMgr@@UAAPAXI@Z 00016d4c f i StateMachineMgr.obj
 0001:00005d7c       ?UpdateStatusFromRIL@CStateMachineMgr@@QAAHXZ 00016d7c f   StateMachineMgr.obj
 0001:00005dd4       ?Check@CStateMachineMgr@@QAAKH@Z 00016dd4 f   StateMachineMgr.obj
 0001:00006290       ??0CUSSDDialog@@QAA@XZ     00017290 f   USSDDialog.obj
 0001:000062b4       ??1CUSSDDialog@@UAA@XZ     000172b4 f   USSDDialog.obj
 0001:000062d8       ?UpdateUSSDData@CUSSDDialog@@QAAXPAUrilsupservicedata_tag@@@Z 000172d8 f   USSDDialog.obj
 0001:00006334       ?ShowWindow@CUSSDDialog@@QAAXH@Z 00017334 f   USSDDialog.obj
 0001:0000634c       ?SetForegroundWindow@CUSSDDialog@@QAAHXZ 0001734c f   USSDDialog.obj
 0001:00006368       ?Initialize@CUSSDDialog@@QAAXXZ 00017368 f   USSDDialog.obj
 0001:00006410       ??_GCUSSDDialog@@UAAPAXI@Z 00017410 f i USSDDialog.obj
 0001:00006410       ??_ECUSSDDialog@@UAAPAXI@Z 00017410 f i USSDDialog.obj
 0001:00006454       ?SetMessageText@CUSSDDialog@@QAAXXZ 00017454 f   USSDDialog.obj
 0001:00006660       ?USSDDialogProc@CUSSDDialog@@SAHPAUHWND__@@IIJ@Z 00017660 f   USSDDialog.obj
 0001:0000684c       ?Create@CUSSDDialog@@QAAHPAUHWND__@@PAUrilsupservicedata_tag@@@Z 0001784c f   USSDDialog.obj
 0001:000069a4       ?Init@CComCriticalSection@ATL@@QAAJXZ 000179a4 f i winmodemstat.obj
 0001:000069fc       ??0CModemStatus@@QAA@XZ    000179fc f   winmodemstat.obj
 0001:00006a54       ?Deregister@CModemStatus@@SAXXZ 00017a54 f   winmodemstat.obj
 0001:00006a80       ?ModReadPDP@CModemStatus@@SAJK@Z 00017a80 f   winmodemstat.obj
 0001:00006a88       ?SetSlotInfo@CModemStatus@@SAHH@Z 00017a88 f   winmodemstat.obj
 0001:00006a90       ?Send2UI@CModemStatus@@SAJIIJ@Z 00017a90 f   winmodemstat.obj
 0001:00006b58       ?UpdateCallTypeAndStatus@CModemStatus@@KAKKKG@Z 00017b58 f   winmodemstat.obj
 0001:00007050       ?ParseDetailErrorCode@CModemStatus@@SAHPAUtagRLE_RILDEVSPECIFIC_ErrorCode@@KG@Z 00018050 f   winmodemstat.obj
 0001:000070c4       ?IsDMMode@CModemStatus@@SAHXZ 000180c4 f   winmodemstat.obj
 0001:000070d4       ??8?$_Const_iterator@$00@?$list@VCResultListElement@@V?$allocator@VCResultListElement@@@std@@@std@@QBA_NABV012@@Z 000180d4 f i winmodemstat.obj
 0001:0000711c       ??E?$_Const_iterator@$00@?$list@VCResultListElement@@V?$allocator@VCResultListElement@@@std@@@std@@QAAAAV012@XZ 0001811c f i winmodemstat.obj
 0001:00007158       ??$_Allocate@U_Node@?$_List_nod@VCResultListElement@@V?$allocator@VCResultListElement@@@std@@@std@@@std@@YAPAU_Node@?$_List_nod@VCResultListElement@@V?$allocator@VCResultListElement@@@std@@@0@IPAU120@@Z 00018158 f i winmodemstat.obj
 0001:000071c8       ??1CModemStatus@@UAA@XZ    000181c8 f   winmodemstat.obj
 0001:000071d8       ??_GCModemStatus@@UAAPAXI@Z 000181d8 f i winmodemstat.obj
 0001:000071d8       ??_ECModemStatus@@UAAPAXI@Z 000181d8 f i winmodemstat.obj
 0001:00007208       ?_Buynode@?$list@VCResultListElement@@V?$allocator@VCResultListElement@@@std@@@std@@IAAPAU_Node@?$_List_nod@VCResultListElement@@V?$allocator@VCResultListElement@@@std@@@2@XZ 00018208 f i winmodemstat.obj
 0001:0000722c       ?_Buynode@?$list@VCResultListElement@@V?$allocator@VCResultListElement@@@std@@@std@@IAAPAU_Node@?$_List_nod@VCResultListElement@@V?$allocator@VCResultListElement@@@std@@@2@PAU342@0ABVCResultListElement@@@Z 0001822c f i winmodemstat.obj
 0001:00007284       ?clear@?$list@VCResultListElement@@V?$allocator@VCResultListElement@@@std@@@std@@QAAXXZ 00018284 f i winmodemstat.obj
 0001:000072dc       ?erase@?$list@VCResultListElement@@V?$allocator@VCResultListElement@@@std@@@std@@QAA?AV?$_Iterator@$00@12@V312@@Z 000182dc f i winmodemstat.obj
 0001:00007374       ?RilResultCallback@CModemStatus@@KAXKJPBXKK@Z 00018374 f   winmodemstat.obj
 0001:00007750       ?_Incsize@?$list@VCResultListElement@@V?$allocator@VCResultListElement@@@std@@@std@@IAAXI@Z 00018750 f i winmodemstat.obj
 0001:000077f8       ?insert@?$list@VCResultListElement@@V?$allocator@VCResultListElement@@@std@@@std@@QAA?AV?$_Iterator@$00@12@V312@ABVCResultListElement@@@Z 000187f8 f i winmodemstat.obj
 0001:00007874       ?AddResultItem@CModemStatus@@KAXJW4eFuncId@CResultListElement@@K@Z 00018874 f   winmodemstat.obj
 0001:00007988       ?ModGetSubscriberNumber@CModemStatus@@SAJXZ 00018988 f   winmodemstat.obj
 0001:00007aa8       ?SendSupServiceData@CModemStatus@@SAJPAGK@Z 00018aa8 f   winmodemstat.obj
 0001:00007ae4       ?CancelSupServiceDataSession@CModemStatus@@SAJXZ 00018ae4 f   winmodemstat.obj
 0001:00007b14       ?ModGetOpState@CModemStatus@@SAJXZ 00018b14 f   winmodemstat.obj
 0001:00007b4c       ?ModGetCallList@CModemStatus@@SAJXZ 00018b4c f   winmodemstat.obj
 0001:00007c80       ?ModGetRegistrationStatus@CModemStatus@@SAJXZ 00018c80 f   winmodemstat.obj
 0001:00007dbc       ?RilNotifyCallback@CModemStatus@@KAXKPBXKK@Z 00018dbc f   winmodemstat.obj
 0001:000081ac       ?Read@CModemStatus@@SAJK@Z 000191ac f   winmodemstat.obj
 0001:00008270       ?ExecNoParamDevSpecific@CModemStatus@@SAJK@Z 00019270 f   winmodemstat.obj
 0001:00008420       ?GetModemTime@CModemStatus@@SAHXZ 00019420 f   winmodemstat.obj
 0001:00008454       ?StartDMMode@CModemStatus@@SAHK@Z 00019454 f   winmodemstat.obj
 0001:000084b8       ?StopDMMode@CModemStatus@@SAHXZ 000194b8 f   winmodemstat.obj
 0001:000084dc       ?StopEmergencyMode@CModemStatus@@SAJXZ 000194dc f   winmodemstat.obj
 0001:00008634       ?Init@CModemStatus@@QAAJPAUHWND__@@@Z 00019634 f   winmodemstat.obj
 0001:000086d8       RIL_Deinitialize           000196d8 f   ril:ril.dll
 0001:000086e8       RIL_GetSubscriberNumbers   000196e8 f   ril:ril.dll
 0001:000086f8       RIL_SendSupServiceData     000196f8 f   ril:ril.dll
 0001:00008708       RIL_CancelSupServiceDataSession 00019708 f   ril:ril.dll
 0001:00008718       RIL_GetEquipmentState      00019718 f   ril:ril.dll
 0001:00008728       RIL_GetCallList            00019728 f   ril:ril.dll
 0001:00008738       RIL_GetRegistrationStatus  00019738 f   ril:ril.dll
 0001:00008748       RIL_DevSpecific            00019748 f   ril:ril.dll
 0001:00008758       RIL_GetSystemTime          00019758 f   ril:ril.dll
 0001:00008768       RIL_Initialize             00019768 f   ril:ril.dll
 0001:00008778       CloseToolhelp32Snapshot    00019778 f   toolhelp:toolhelp.dll
 0001:00008788       Process32Next              00019788 f   toolhelp:toolhelp.dll
 0001:00008798       Process32First             00019798 f   toolhelp:toolhelp.dll
 0001:000087a8       CreateToolhelp32Snapshot   000197a8 f   toolhelp:toolhelp.dll
 0001:000087b8       Sleep                      000197b8 f   coredll:COREDLL.dll
 0001:000087c8       FindClose                  000197c8 f   coredll:COREDLL.dll
 0001:000087d8       FindFirstFileW             000197d8 f   coredll:COREDLL.dll
 0001:000087e8       WaitForSingleObject        000197e8 f   coredll:COREDLL.dll
 0001:000087f8       wcscpy                     000197f8 f   coredll:COREDLL.dll
 0001:00008808       GetLastError               00019808 f   coredll:COREDLL.dll
 0001:00008818       LoadLibraryW               00019818 f   coredll:COREDLL.dll
 0001:00008828       CreateMutexW               00019828 f   coredll:COREDLL.dll
 0001:00008838       GetMessageW                00019838 f   coredll:COREDLL.dll
 0001:00008848       DispatchMessageW           00019848 f   coredll:COREDLL.dll
 0001:00008858       TranslateMessage           00019858 f   coredll:COREDLL.dll
 0001:00008868       wcsrchr                    00019868 f   coredll:COREDLL.dll
 0001:00008878       EventModify                00019878 f   coredll:COREDLL.dll
 0001:00008888       ??3@YAXPAX@Z               00019888 f   coredll:COREDLL.dll
 0001:00008898       CreateEventW               00019898 f   coredll:COREDLL.dll
 0001:000088a8       InitializeCriticalSection  000198a8 f   coredll:COREDLL.dll
 0001:000088b8       ??2@YAPAXI@Z               000198b8 f   coredll:COREDLL.dll
 0001:000088c8       _wcsicmp                   000198c8 f   coredll:COREDLL.dll
 0001:000088d8       CloseHandle                000198d8 f   coredll:COREDLL.dll
 0001:000088e8       DeleteCriticalSection      000198e8 f   coredll:COREDLL.dll
 0001:000088f8       LeaveCriticalSection       000198f8 f   coredll:COREDLL.dll
 0001:00008908       EnterCriticalSection       00019908 f   coredll:COREDLL.dll
 0001:00008918       NKDbgPrintfW               00019918 f   coredll:COREDLL.dll
 0001:00008928       CreateThread               00019928 f   coredll:COREDLL.dll
 0001:00008938       MessageBoxW                00019938 f   coredll:COREDLL.dll
 0001:00008948       LoadStringW                00019948 f   coredll:COREDLL.dll
 0001:00008958       CreateProcessW             00019958 f   coredll:COREDLL.dll
 0001:00008968       SystemIdleTimerReset       00019968 f   coredll:COREDLL.dll
 0001:00008978       PostMessageW               00019978 f   coredll:COREDLL.dll
 0001:00008988       RegisterWindowMessageW     00019988 f   coredll:COREDLL.dll
 0001:00008998       SetDlgItemTextW            00019998 f   coredll:COREDLL.dll
 0001:000089a8       wsprintfW                  000199a8 f   coredll:COREDLL.dll
 0001:000089b8       ShowWindow                 000199b8 f   coredll:COREDLL.dll
 0001:000089c8       SetForegroundWindow        000199c8 f   coredll:COREDLL.dll
 0001:000089d8       memset                     000199d8 f   coredll:COREDLL.dll
 0001:000089e8       GetWindowLongW             000199e8 f   coredll:COREDLL.dll
 0001:000089f8       DestroyWindow              000199f8 f   coredll:COREDLL.dll
 0001:00008a08       EnableWindow               00019a08 f   coredll:COREDLL.dll
 0001:00008a18       GetDlgItem                 00019a18 f   coredll:COREDLL.dll
 0001:00008a28       SetWindowLongW             00019a28 f   coredll:COREDLL.dll
 0001:00008a38       CreateDialogIndirectParamW 00019a38 f   coredll:COREDLL.dll
 0001:00008a48       LoadResource               00019a48 f   coredll:COREDLL.dll
 0001:00008a58       FindResourceW              00019a58 f   coredll:COREDLL.dll
 0001:00008a68       KillTimer                  00019a68 f   coredll:COREDLL.dll
 0001:00008a78       LoadImageW                 00019a78 f   coredll:COREDLL.dll
 0001:00008a88       SetTimer                   00019a88 f   coredll:COREDLL.dll
 0001:00008a98       RegCloseKey                00019a98 f   coredll:COREDLL.dll
 0001:00008aa8       RegSetValueExW             00019aa8 f   coredll:COREDLL.dll
 0001:00008ab8       RegQueryValueExW           00019ab8 f   coredll:COREDLL.dll
 0001:00008ac8       RegOpenKeyExW              00019ac8 f   coredll:COREDLL.dll
 0001:00008ad8       wcscmp                     00019ad8 f   coredll:COREDLL.dll
 0001:00008ae8       wcsncpy                    00019ae8 f   coredll:COREDLL.dll
 0001:00008af8       wcslen                     00019af8 f   coredll:COREDLL.dll
 0001:00008b08       RasEnumConnections         00019b08 f   coredll:COREDLL.dll
 0001:00008b18       SetSystemTime              00019b18 f   coredll:COREDLL.dll
 0001:00008b28       memcpy                     00019b28 f   coredll:COREDLL.dll
 0001:00008b38       RegisterClassW             00019b38 f   coredll:COREDLL.dll
 0001:00008b48       GetStockObject             00019b48 f   coredll:COREDLL.dll
 0001:00008b58       LoadIconW                  00019b58 f   coredll:COREDLL.dll
 0001:00008b68       CreateWindowExW            00019b68 f   coredll:COREDLL.dll
 0001:00008b78       DefWindowProcW             00019b78 f   coredll:COREDLL.dll
 0001:00008b88       SetWindowTextW             00019b88 f   coredll:COREDLL.dll
 0001:00008b98       BringWindowToTop           00019b98 f   coredll:COREDLL.dll
 0001:00008ba8       strlen                     00019ba8 f   coredll:COREDLL.dll
 0001:00008bb8       ??0exception@std@@QAA@PBD@Z 00019bb8 f   coredll:COREDLL.dll
 0001:00008bc8       ?what@exception@std@@UBAPBDXZ 00019bc8 f   coredll:COREDLL.dll
 0001:00008bd8       ??1exception@std@@UAA@XZ   00019bd8 f   coredll:COREDLL.dll
 0001:00008be8       __CxxThrowException        00019be8 f   coredll:COREDLL.dll
 0001:00008bf8       ??_7type_info@@6B@         00019bf8 f   coredll:COREDLL.dll
 0001:00008c08       ??0exception@std@@QAA@ABV01@@Z 00019c08 f   coredll:COREDLL.dll
 0001:00008c18       ??0exception@std@@QAA@XZ   00019c18 f   coredll:COREDLL.dll
 0001:00008c28       RasHangUp                  00019c28 f   coredll:COREDLL.dll
 0001:00008c38       RasGetConnectStatus        00019c38 f   coredll:COREDLL.dll
 0001:00008c48       FindWindowW                00019c48 f   coredll:COREDLL.dll
 0001:00008c58       ??_U@YAPAXI@Z              00019c58 f   coredll:COREDLL.dll
 0001:00008c68       wcscat                     00019c68 f   coredll:COREDLL.dll
 0001:00008c78       GetDlgItemTextW            00019c78 f   coredll:COREDLL.dll
 0001:00008c88       RaiseException             00019c88 f   coredll:COREDLL.dll
 0001:00008c98       __C_specific_handler       00019c98 f   coredll:COREDLL.dll
 0001:00008ca8       SendMessageTimeout         00019ca8 f   coredll:COREDLL.dll
 0001:00008cb8       free                       00019cb8 f   coredll:COREDLL.dll
 0001:00008cc8       TerminateProcess           00019cc8 f   coredll:COREDLL.dll
 0001:00008cd8       ??_V@YAXPAX@Z              00019cd8 f   coredll:COREDLL.dll
 0001:00008ce8       ExitWindowsEx              00019ce8 f   aygshell:AYGSHELL.dll
 0001:00008cf8       SHInitDialog               00019cf8 f   aygshell:AYGSHELL.dll
 0001:00008d08       SHCreateMenuBar            00019d08 f   aygshell:AYGSHELL.dll
 0001:00008d18       SHNotificationAdd          00019d18 f   aygshell:AYGSHELL.dll
 0001:00008d28       SHNotificationRemove       00019d28 f   aygshell:AYGSHELL.dll
 0001:00008d38       SHNotificationUpdate       00019d38 f   aygshell:AYGSHELL.dll
 0001:00008d48       SHNotificationGetData      00019d48 f   aygshell:AYGSHELL.dll
 0001:00008d58       SHEnableSoftkey            00019d58 f   aygshell:AYGSHELL.dll
 0001:00008d70       WinMainCRTStartup          00019d70 f   corelibc:pegwmain.obj
 0001:00008de4       __security_check_cookie    00019de4     corelibc:armsecgs.obj
 0001:00008df8       __gsfailure                00019df8     corelibc:armsecgs.obj
 0001:00008e3c       _onexit                    00019e3c f   corelibc:onexit.obj
 0001:00008ee8       atexit                     00019ee8 f   corelibc:onexit.obj
 0001:00008f08       _cinit                     00019f08 f   corelibc:crt0dat.obj
 0001:00009078       exit                       0001a078 f   corelibc:crt0dat.obj
 0001:00009090       __security_init_cookie     0001a090 f   corelibc:seccinit.obj
 0001:000090e0       ??1out_of_range@std@@UAA@XZ 0001a0e0 f i libcpmt:string.obj
 0001:0000910c       ??_Gout_of_range@std@@UAAPAXI@Z 0001a10c f i libcpmt:string.obj
 0001:0000910c       ??_Eout_of_range@std@@UAAPAXI@Z 0001a10c f i libcpmt:string.obj
 0001:00009160       ?_Xlen@_String_base@std@@SAXXZ 0001a160 f   libcpmt:string.obj
 0001:000091f0       ?_Xran@_String_base@std@@SAXXZ 0001a1f0 f   libcpmt:string.obj
 0001:00009278       ??0out_of_range@std@@QAA@ABV01@@Z 0001a278 f i libcpmt:string.obj
 0001:000092b0       __FrameUnwindToState       0001a2b0 f   LIBCMT:frame_ce.obj
 0001:00009628       ?_DestructExceptionObject@@YAXPAUEHExceptionRecord@@E@Z 0001a628 f   LIBCMT:frame_ce.obj
 0001:00009694       ?_OffsetToAddress@@YAPAXHPAKK@Z 0001a694 f   LIBCMT:frame_ce.obj
 0001:000096e0       ?FindFrameInfo@@YAPAU_FrameInfo@@PAK@Z 0001a6e0 f   LIBCMT:frame_ce.obj
 0001:00009720       ?FindCatchFrameInfo@@YAPAU_FrameInfo@@PAK@Z 0001a720 f   LIBCMT:frame_ce.obj
 0001:00009760       ?_GetRangeOfTrysToCheck@@YAPBU_s_TryBlockMapEntry@@PBU_s_FuncInfo@@HHPAI1@Z 0001a760 f   LIBCMT:frame_ce.obj
 0001:0000a16c       __InternalCxxFrameHandler  0001b16c f   LIBCMT:frame_ce.obj
 0001:0000a2c4       __CxxFrameHandler3         0001b2c4 f   LIBCMT:frame_ce.obj
 0001:0000a2fc       __GSHandlerCheckCommon     0001b2fc f   LIBCMT:gshandler.obj
 0001:0000a344       __GSHandlerCheck           0001b344 f   LIBCMT:gshandler.obj
 0001:0000a374       memcpy_s                   0001b374 f   LIBCMT:memcpy_s.obj
 0001:0000a45c       memmove_s                  0001b45c f   LIBCMT:memmove_s.obj
 0001:0000a514       _invalid_parameter_noinfo  0001b514 f   LIBCMT:invarg.obj
 0001:0000a550       _invoke_watson             0001b550 f   LIBCMT:invarg.obj
 0001:0000a57c       __GSHandlerCheck_EH        0001b57c f   LIBCMT:gshandlereh.obj
 0001:0000a610       GetCRTStorage              0001b610 f   LIBCMT:corecrt.obj
 0001:0000a6dc       _CallSettingFrame          0001b6dc     LIBCMT:handlers_arm.obj
 0001:0000a720       ?FindFrameForUnwind@@YAPAKPAKPBU_s_FuncInfo@@@Z 0001b720 f   LIBCMT:mdframe_arm.obj
 0001:0000a768       ?FindCatchFrame@@YAPAKPAKK@Z 0001b768 f   LIBCMT:mdframe_arm.obj
 0001:0000a7b4       ?AdjustFrameForCatch@@YAPAKPAKPBU_s_FuncInfo@@@Z 0001b7b4 f   LIBCMT:mdframe_arm.obj
 0001:0000a7ec       ?GetCurrentState@@YAHPAKPAU_DISPATCHER_CONTEXT@@PBU_s_FuncInfo@@@Z 0001b7ec f   LIBCMT:ehstate_arm_mips.obj
 0001:0000a848       _invalid_parameter         0001b848 f   LIBCMT:invarginternal.obj
 0001:0000a874       AtlRawDllMain              0001b874 f   atls:atlbase.obj
 0001:0000a90c       ?RemoveAll@?$CSimpleArray@PAUHINSTANCE__@@V?$CSimpleArrayEqualHelper@PAUHINSTANCE__@@@ATL@@@ATL@@QAAXXZ 0001b90c f i atls:atlbase.obj
 0001:0000a948       ??0_ATL_BASE_MODULE70@ATL@@QAA@XZ 0001b948 f i atls:atlbase.obj
 0001:0000a98c       ??1CAtlBaseModule@ATL@@QAA@XZ 0001b98c f   atls:atlbase.obj
 0001:0000a9c4       ??0CAtlBaseModule@ATL@@QAA@XZ 0001b9c4 f   atls:atlbase.obj
 0001:0000aa60       _XcptFilter                0001ba60 f   coredll:COREDLL.dll
 0001:0000aa70       __report_gsfailure         0001ba70 f   coredll:COREDLL.dll
 0001:0000aa80       LocalReAlloc               0001ba80 f   coredll:COREDLL.dll
 0001:0000aa90       LocalAlloc                 0001ba90 f   coredll:COREDLL.dll
 0001:0000aaa0       LocalSize                  0001baa0 f   coredll:COREDLL.dll
 0001:0000aab0       LocalFree                  0001bab0 f   coredll:COREDLL.dll
 0001:0000aac0       __security_gen_cookie      0001bac0 f   coredll:COREDLL.dll
 0001:0000aad0       strcmp                     0001bad0 f   coredll:COREDLL.dll
 0001:0000aae0       ?terminate@std@@YAXXZ      0001bae0 f   coredll:COREDLL.dll
 0001:0000aaf0       memmove                    0001baf0 f   coredll:COREDLL.dll
 0001:0000ab00       TlsCall                    0001bb00 f   coredll:COREDLL.dll
 0001:0000ab10       TlsSetValue                0001bb10 f   coredll:COREDLL.dll
 0001:0000ab20       TlsGetValue                0001bb20 f   coredll:COREDLL.dll
 0001:0000ab30       InterlockedCompareExchange 0001bb30 f   coredll:COREDLL.dll
 0001:0000ab40       GetModuleHandleW           0001bb40 f   coredll:COREDLL.dll
 0002:00000000       ??_C@_0P@GHFPNOJB@bad?5allocation?$AA@ 0001d000     AAM.obj
 0002:0000004c       ??_C@_1DK@IMJIOKDD@?$AA?2?$AAW?$AAi?$AAn?$AAd?$AAo?$AAw?$AAs?$AA?2?$AAS?$AAt?$AAa?$AAr?$AAt?$AAU?$AAp?$AA?2?$AAW?$AAe?$AAl?$AAc?$AAo?$AAm?$AAe?$AA?4?$AAl?$AAn?$AAk?$AA?$AA@ 0001d04c     AAM.obj
 0002:000000bc       ??_7CAAMApp@@6B@           0001d0bc     AAM.obj
 0002:000000c4       ??_C@_1CM@PGIJNMC@?$AAC?$AAo?$AAn?$AAn?$AAe?$AAc?$AAt?$AAi?$AAo?$AAn?$AAP?$AAr?$AAo?$AAf?$AAi?$AAl?$AAe?$AAN?$AAa?$AAm?$AAe?$AA?$AA@ 0001d0c4     AAM.obj
 0002:000000f0       ??_C@_11LOCGONAA@?$AA?$AA@ 0001d0f0     AAM.obj
 0002:000000f4       ??_C@_1BO@BMNAGPCC@?$AAA?$AAi?$AAr?$AAp?$AAr?$AAi?$AAm?$AAe?$AA?5?$AAM?$AAo?$AAd?$AAe?$AAm?$AA?$AA@ 0001d0f4     AAM.obj
 0002:00000114       ??_C@_1BE@BFGEGPNA@?$AAM?$AAo?$AAd?$AAe?$AAm?$AAN?$AAa?$AAm?$AAe?$AA?$AA@ 0001d114     AAM.obj
 0002:00000128       ??_C@_1BE@CEBCAMKF@?$AA?4?$AA?2?$AAa?$AAa?$AAm?$AA?4?$AAc?$AAp?$AAp?$AA?$AA@ 0001d128     AAM.obj
 0002:0000013c       ??_C@_1DO@GNDAEGEA@?$AAL?$AAo?$AAa?$AAd?$AAL?$AAi?$AAb?$AAr?$AAa?$AAr?$AAy?$AA?5?$AA?$CF?$AAs?$AA?5?$AAf?$AAa?$AAi?$AAl?$AAe?$AAd?$AA?5?$AAe?$AAr?$AAr?$AAo?$AAr?$AA?5?$AA?$CF?$AAd?$AA?$AA@ 0001d13c     AAM.obj
 0002:0000017c       ??_C@_1CA@MNHLNOBN@?$AAs?$AAw?$AAi?$AA_?$AAr?$AAi?$AAl?$AAr?$AAe?$AAs?$AAG?$AA?4?$AAd?$AAl?$AAl?$AA?$AA@ 0001d17c     AAM.obj
 0002:0000019c       ??_C@_1CA@DGCLHOME@?$AAA?$AAA?$AAM?$AAM?$AAu?$AAt?$AAe?$AAx?$AA?5?$AAo?$AAf?$AA?5?$AAS?$AAW?$AAI?$AA?$AA@ 0001d19c     AAM.obj
 0002:00000210       ??_7CArbitrator@@6B@       0001d210     Arbitrator.obj
 0002:00000218       ??_C@_1BG@JEMNDGK@?$AAS?$AAP?$AAI?$AAD?$AAE?$AAR?$AA?4?$AAE?$AAX?$AAE?$AA?$AA@ 0001d218     Arbitrator.obj
 0002:00000230       ??_C@_1EK@MEIPNALP@?$AAC?$AAr?$AAe?$AAa?$AAt?$AAe?$AAT?$AAo?$AAo?$AAl?$AAh?$AAe?$AAl?$AAp?$AA3?$AA2?$AAS?$AAn?$AAa?$AAp?$AAs?$AAh?$AAo?$AAt?$AA?5?$AAf?$AAa?$AAi?$AAl?$AAe?$AAd?$AA?5@ 0001d230     Arbitrator.obj
 0002:0000027c       ??_C@_1DG@LDDFKNGI@?$AAP?$AAr?$AAo?$AAc?$AAe?$AAs?$AAs?$AA3?$AA2?$AAF?$AAi?$AAr?$AAs?$AAt?$AA?5?$AAf?$AAa?$AAi?$AAl?$AAe?$AAd?$AA?5?$AA?$CF?$AAl?$AAu?$AA?6?$AA?$AA@ 0001d27c     Arbitrator.obj
 0002:000002b4       ??_C@_1DE@MNBDLDPM@?$AAP?$AAr?$AAo?$AAc?$AAe?$AAs?$AAs?$AA3?$AA2?$AAN?$AAe?$AAx?$AAt?$AA?5?$AAf?$AAa?$AAi?$AAl?$AAe?$AAd?$AA?5?$AA?$CF?$AAl?$AAu?$AA?6?$AA?$AA@ 0001d2b4     Arbitrator.obj
 0002:000002e8       ??_C@_1GM@PKEFHHO@?$AAU?$AAn?$AAa?$AAb?$AAl?$AAe?$AA?5?$AAt?$AAo?$AA?5?$AAs?$AAt?$AAa?$AAr?$AAt?$AA?5?$AAC?$AAl?$AAi?$AAe?$AAn?$AAt?$AA?5?$AAI?$AAn?$AAi?$AAt?$AAi?$AAa?$AAt?$AAe?$AAd@ 0001d2e8     Arbitrator.obj
 0002:00000354       ??_C@_17MONHFMNG@?$AAp?$AAd?$AAp?$AA?$AA@ 0001d354     Arbitrator.obj
 0002:0000035c       ??_C@_1CC@LEFEIIAN@?$AA?4?$AA?2?$AAa?$AAr?$AAb?$AAi?$AAt?$AAr?$AAa?$AAt?$AAo?$AAr?$AA?4?$AAc?$AAp?$AAp?$AA?$AA@ 0001d35c     Arbitrator.obj
 0002:00000380       ??_C@_1FM@OPEKIPPJ@?$AAU?$AAn?$AAa?$AAb?$AAl?$AAe?$AA?5?$AAt?$AAo?$AA?5?$AAs?$AAt?$AAa?$AAr?$AAt?$AA?5?$AAD?$AAe?$AAf?$AAe?$AAr?$AAr?$AAe?$AAd?$AA?5?$AAP?$AAr?$AAo?$AAv?$AAi?$AAs?$AAi@ 0001d380     Arbitrator.obj
 0002:000003dc       ??_C@_17DEMEBEPH@?$AAa?$AAa?$AAl?$AA?$AA@ 0001d3dc     Arbitrator.obj
 0002:000003e4       ??_C@_1DI@GBDICIOO@?$AA?2?$AAW?$AAi?$AAn?$AAd?$AAo?$AAw?$AAs?$AA?2?$AAI?$AAO?$AAT?$AAA?$AAT?$AAh?$AAi?$AAn?$AAC?$AAl?$AAi?$AAe?$AAn?$AAt?$AA?4?$AAe?$AAx?$AAe?$AA?$AA@ 0001d3e4     Arbitrator.obj
 0002:0000041c       ??_C@_1CG@MBJAPMKG@?$AAI?$AAO?$AAT?$AAA?$AAT?$AAh?$AAi?$AAn?$AAC?$AAl?$AAi?$AAe?$AAn?$AAt?$AA?4?$AAe?$AAx?$AAe?$AA?$AA@ 0001d41c     Arbitrator.obj
 0002:00000444       ??_C@_1CI@GLJPOLKK@?$AAc?$AAa?$AAn?$AA?8?$AAt?$AA?5?$AAL?$AAa?$AAu?$AAn?$AAc?$AAh?$AA?5?$AAA?$AAc?$AAt?$AAW?$AAi?$AAz?$AA?$AA@ 0001d444     Arbitrator.obj
 0002:0000046c       ??_C@_1CI@JIKPJHIB@?$AA?2?$AAW?$AAi?$AAn?$AAd?$AAo?$AAw?$AAs?$AA?2?$AAA?$AAc?$AAt?$AAW?$AAi?$AAz?$AA?4?$AAe?$AAx?$AAe?$AA?$AA@ 0001d46c     Arbitrator.obj
 0002:00000494       ??_C@_1BE@CENHHBC@?$AAI?$AAT?$AAO?$AAA?$AA_?$AAE?$AAX?$AAI?$AAT?$AA?$AA@ 0001d494     Arbitrator.obj
 0002:000004a8       ??_7CIota24Dlg@@6B@        0001d4a8     iota24dlg.obj
 0002:00000618       ??_7CMainFrame@@6B@        0001d618     MainFrm.obj
 0002:00000770       ??_C@_1GC@MBPIJLDO@?$AAC?$AAM?$AAa?$AAi?$AAn?$AAF?$AAr?$AAa?$AAm?$AAe?$AA?3?$AA?3?$AAR?$AAe?$AAm?$AAo?$AAv?$AAe?$AAW?$AAP?$AAS?$AAB?$AAu?$AAb?$AAb?$AAl?$AAe?$AA?3?$AA?5?$AAW?$AAP?$AAS@ 0001d770     MainFrm.obj
 0002:000007d4       ??_C@_1BM@HGFEFMNP@?$AA?4?$AA?2?$AAm?$AAa?$AAi?$AAn?$AAf?$AAr?$AAm?$AA?4?$AAc?$AAp?$AAp?$AA?$AA@ 0001d7d4     MainFrm.obj
 0002:000007f0       ??_C@_1IO@CCIGLPH@?$AAC?$AAM?$AAa?$AAi?$AAn?$AAF?$AAr?$AAa?$AAm?$AAe?$AA?3?$AA?3?$AAI?$AAn?$AAs?$AAe?$AAr?$AAt?$AAW?$AAP?$AAS?$AAB?$AAu?$AAb?$AAb?$AAl?$AAe?$AA?3?$AA?5?$AAU?$AAn?$AAa@ 0001d7f0     MainFrm.obj
 0002:00000880       ??_C@_19MBCBCBDA@?$AAH?$AAi?$AAd?$AAe?$AA?$AA@ 0001d880     MainFrm.obj
 0002:0000088c       ??_C@_1BA@IHNFGJPH@?$AAD?$AAi?$AAs?$AAm?$AAi?$AAs?$AAs?$AA?$AA@ 0001d88c     MainFrm.obj
 0002:000008a0       ??_C@_1GA@OOGCDGEG@?$AAC?$AAM?$AAa?$AAi?$AAn?$AAF?$AAr?$AAa?$AAm?$AAe?$AA?3?$AA?3?$AAR?$AAe?$AAm?$AAo?$AAv?$AAe?$AAW?$AAP?$AAS?$AAB?$AAu?$AAb?$AAb?$AAl?$AAe?$AA?3?$AA?5?$AAW?$AAP?$AAS@ 0001d8a0     MainFrm.obj
 0002:00000900       ??_C@_1JE@BGKGOEOO@?$AAC?$AAM?$AAa?$AAi?$AAn?$AAF?$AAr?$AAa?$AAm?$AAe?$AA?3?$AA?3?$AAR?$AAe?$AAm?$AAo?$AAv?$AAe?$AAW?$AAP?$AAS?$AAB?$AAu?$AAb?$AAb?$AAl?$AAe?$AA?3?$AA?5?$AAU?$AAn?$AAa@ 0001d900     MainFrm.obj
 0002:00000998       ??_C@_1FG@NAKOENC@?$AAS?$AAH?$AAN?$AAo?$AAt?$AAi?$AAf?$AAi?$AAc?$AAa?$AAt?$AAi?$AAo?$AAn?$AAG?$AAe?$AAt?$AAD?$AAa?$AAt?$AAa?$AA?5?$AAf?$AAa?$AAi?$AAl?$AAe?$AAd?$AA?5?$AAw?$AAi?$AAt@ 0001d998     MainFrm.obj
 0002:000009f0       ??_C@_1FE@IPKCHHMO@?$AAS?$AAH?$AAN?$AAo?$AAt?$AAi?$AAf?$AAi?$AAc?$AAa?$AAt?$AAi?$AAo?$AAn?$AAU?$AAp?$AAd?$AAa?$AAt?$AAe?$AA?5?$AAf?$AAa?$AAi?$AAl?$AAe?$AAd?$AA?5?$AAw?$AAi?$AAt?$AAh@ 0001d9f0     MainFrm.obj
 0002:00000a44       ??_C@_1O@JBBHAGJJ@?$AA?$CF?$AAs?$AA?$CF?$AAs?$AA?$CF?$AAs?$AA?$AA@ 0001da44     MainFrm.obj
 0002:00000a58       ??_C@_1FA@EHANOMAP@?$AAF?$AAa?$AAi?$AAl?$AA?5?$AAt?$AAo?$AA?5?$AAi?$AAn?$AAs?$AAe?$AAr?$AAt?$AA?5?$AAe?$AAm?$AAe?$AAr?$AAg?$AAe?$AAn?$AAc?$AAy?$AA?5?$AAi?$AAc?$AAo?$AAn?$AA?5?$AAl?$AAR@ 0001da58     MainFrm.obj
 0002:00000aa8       ??_C@_1GG@JOAPJPLB@?$AAM?$AAD?$AAN?$AA?5?$AAf?$AAr?$AAo?$AAm?$AA?5?$AAm?$AAo?$AAd?$AAe?$AAm?$AA?5?$AAi?$AAs?$AA?5?$AAp?$AAo?$AAi?$AAn?$AAt?$AAe?$AAr?$AA?5?$AA?$DN?$AA?5?$AA?$CF?$AAp?$AA?5?$AAo@ 0001daa8     MainFrm.obj
 0002:00000b10       ??_C@_1HE@KMOGMNJM@?$AAA?$AAA?$AAM?$AA?3?$AA?5?$AAF?$AAa?$AAi?$AAl?$AAe?$AAd?$AA?5?$AAt?$AAo?$AA?5?$AAr?$AAe?$AAa?$AAd?$AA?5?$AAc?$AAa?$AAl?$AAl?$AAb?$AAa?$AAc?$AAk?$AA?5?$AAn?$AAu?$AAm@ 0001db10     MainFrm.obj
 0002:00000b88       ??_C@_1HC@CJJJDMPA@?$AAA?$AAA?$AAM?$AA?3?$AA?5?$AAF?$AAa?$AAi?$AAl?$AAe?$AAd?$AA?5?$AAt?$AAo?$AA?5?$AAw?$AAr?$AAi?$AAt?$AAe?$AA?5?$AAc?$AAa?$AAl?$AAl?$AAb?$AAa?$AAc?$AAk?$AA?5?$AAn?$AAu@ 0001db88     MainFrm.obj
 0002:00000bfc       ??_C@_1CE@FNJMHKND@?$AAS?$AAM?$AAS?$AAC?$AAa?$AAl?$AAl?$AAb?$AAa?$AAc?$AAk?$AAN?$AAu?$AAm?$AAb?$AAe?$AAr?$AA?$AA@ 0001dbfc     MainFrm.obj
 0002:00000c20       ??_C@_1EE@OGJCHBOA@?$AAS?$AAo?$AAf?$AAt?$AAw?$AAa?$AAr?$AAe?$AA?2?$AAM?$AAi?$AAc?$AAr?$AAo?$AAs?$AAo?$AAf?$AAt?$AA?2?$AAI?$AAn?$AAb?$AAo?$AAx?$AA?2?$AAS?$AAe?$AAt?$AAt?$AAi?$AAn?$AAg@ 0001dc20     MainFrm.obj
 0002:00000c68       ??_C@_1GK@PELGFGPO@?$AAU?$AAn?$AAa?$AAb?$AAl?$AAe?$AA?5?$AAt?$AAo?$AA?5?$AAo?$AAp?$AAe?$AAn?$AA?5?$AAt?$AAh?$AAe?$AA?5?$AAr?$AAe?$AAg?$AAi?$AAs?$AAt?$AAr?$AAy?$AA?5?$AAk?$AAe?$AAy?$AA?5@ 0001dc68     MainFrm.obj
 0002:00000cd4       ??_C@_1CO@KNALKICG@?$AAC?$AAa?$AAr?$AAr?$AAi?$AAe?$AAr?$AAP?$AAr?$AAo?$AAv?$AAi?$AAd?$AAe?$AAr?$AAN?$AAu?$AAm?$AAb?$AAe?$AAr?$AA1?$AA?$AA@ 0001dcd4     MainFrm.obj
 0002:00000d04       ??_C@_17MPACHMLF@?$AA?$CK?$AA8?$AA6?$AA?$AA@ 0001dd04     MainFrm.obj
 0002:00000d10       ??_C@_1EK@IEBPLGNP@?$AAU?$AAn?$AAa?$AAb?$AAl?$AAe?$AA?5?$AAQ?$AAu?$AAe?$AAr?$AAy?$AA?5?$AAP?$AAh?$AAo?$AAn?$AAe?$AAN?$AAu?$AAm?$AAb?$AAe?$AAr?$AA1?$AA?5?$AAe?$AAr?$AAr?$AAo?$AAr?$AA?5@ 0001dd10     MainFrm.obj
 0002:00000d60       ??_C@_1HG@HFLEKGCO@?$AAA?$AAA?$AAM?$AA?3?$AA?5?$AAM?$AAD?$AAN?$AA?5?$AAf?$AAr?$AAo?$AAm?$AA?5?$AAt?$AAh?$AAe?$AA?5?$AAr?$AAe?$AAg?$AAi?$AAs?$AAt?$AAr?$AAy?$AA?5?$AAi?$AAs?$AA?5?$AA?$CF?$AAs@ 0001dd60     MainFrm.obj
 0002:00000dd8       ??_C@_13COJANIEC@?$AA0?$AA?$AA@ 0001ddd8     MainFrm.obj
 0002:00000ddc       ??_C@_1BK@KLDAHGN@?$AAP?$AAh?$AAo?$AAn?$AAe?$AAN?$AAu?$AAm?$AAb?$AAe?$AAr?$AA1?$AA?$AA@ 0001dddc     MainFrm.obj
 0002:00000df8       ??_C@_1DC@GDOPCOAK@?$AAS?$AAo?$AAf?$AAt?$AAw?$AAa?$AAr?$AAe?$AA?2?$AAM?$AAi?$AAc?$AAr?$AAo?$AAs?$AAo?$AAf?$AAt?$AA?2?$AAV?$AAm?$AAa?$AAi?$AAl?$AA?$AA@ 0001ddf8     MainFrm.obj
 0002:00000e30       ??_C@_1HE@BMGCCCAC@?$AAC?$AAM?$AAa?$AAi?$AAn?$AAF?$AAr?$AAa?$AAm?$AAe?$AA?3?$AA?3?$AAO?$AAn?$AAR?$AAe?$AAs?$AAu?$AAl?$AAt?$AAG?$AAe?$AAt?$AAM?$AAi?$AAn?$AAA?$AAc?$AAt?$AAi?$AAv?$AAe@ 0001de30     MainFrm.obj
 0002:00000ea4       ??_C@_1DC@PJNNAEJG@?$AAG?$AAe?$AAt?$AAV?$AAe?$AAr?$AAs?$AAi?$AAo?$AAn?$AAI?$AAn?$AAf?$AAo?$AA?5?$AAF?$AAA?$AAI?$AAL?$AAE?$AAD?$AA?$CB?$AA?$CB?$AA?$CB?$AA?$AA@ 0001dea4     MainFrm.obj
 0002:00000ed8       ??_C@_1HK@CLDJAGPA@?$AAA?$AAu?$AAt?$AAo?$AA?5?$AAl?$AAa?$AAu?$AAn?$AAc?$AAh?$AA?5?$AAo?$AAf?$AA?5?$AAG?$AAo?$AAb?$AAi?$AAA?$AAc?$AAt?$AAi?$AAv?$AAa?$AAt?$AAi?$AAo?$AAn?$AA?5?$AAi?$AAs@ 0001ded8     MainFrm.obj
 0002:00000f58       ??_C@_1GI@EMAAFDEH@?$AAF?$AAa?$AAi?$AAl?$AAe?$AAd?$AA?5?$AAt?$AAo?$AA?5?$AAr?$AAe?$AAa?$AAd?$AA?5?$AAN?$AAe?$AAt?$AAw?$AAo?$AAr?$AAk?$AAT?$AAy?$AAp?$AAe?$AA?5?$AAr?$AAe?$AAg?$AAi?$AAs@ 0001df58     MainFrm.obj
 0002:00000fc0       ??_C@_1GK@LHDFOGNN@?$AAG?$AAo?$AAb?$AAi?$AAA?$AAc?$AAt?$AAi?$AAv?$AAa?$AAt?$AAi?$AAo?$AAn?$AA?5?$AAi?$AAs?$AA?5?$AAn?$AAo?$AAt?$AA?5?$AAs?$AAu?$AAp?$AAp?$AAo?$AAr?$AAt?$AAe?$AAd?$AA?5@ 0001dfc0     MainFrm.obj
 0002:00001030       ??_C@_1EC@DHBKNDOP@?$AAU?$AAn?$AAa?$AAb?$AAl?$AAe?$AA?5?$AAt?$AAo?$AA?5?$AAL?$AAa?$AAu?$AAn?$AAc?$AAh?$AA?5?$AAG?$AAo?$AAb?$AAi?$AA?5?$AAA?$AAc?$AAt?$AAi?$AAv?$AAa?$AAt?$AAi?$AAo?$AAn@ 0001e030     MainFrm.obj
 0002:00001074       ??_C@_1DI@LFPNANLM@?$AA?2?$AAW?$AAi?$AAn?$AAd?$AAo?$AAw?$AAs?$AA?2?$AAG?$AAo?$AAb?$AAi?$AAa?$AAc?$AAt?$AAi?$AAv?$AAa?$AAt?$AAi?$AAo?$AAn?$AA?4?$AAe?$AAx?$AAe?$AA?$AA@ 0001e074     MainFrm.obj
 0002:000010ac       ??_C@_1BI@FJLDDKCH@?$AAN?$AAe?$AAt?$AAw?$AAo?$AAr?$AAk?$AAT?$AAy?$AAp?$AAe?$AA?$AA@ 0001e0ac     MainFrm.obj
 0002:000010c4       ??_C@_1CO@PFFMHNAH@?$AAS?$AAo?$AAf?$AAt?$AAw?$AAa?$AAr?$AAe?$AA?2?$AAM?$AAi?$AAc?$AAr?$AAo?$AAs?$AAo?$AAf?$AAt?$AA?2?$AAR?$AAI?$AAL?$AA?$AA@ 0001e0c4     MainFrm.obj
 0002:000010f8       ??_C@_1HM@NMNHLACG@?$AAC?$AAM?$AAa?$AAi?$AAn?$AAF?$AAr?$AAa?$AAm?$AAe?$AA?3?$AA?3?$AAO?$AAn?$AAR?$AAe?$AAs?$AAu?$AAl?$AAt?$AAG?$AAe?$AAt?$AAM?$AAi?$AAn?$AAA?$AAc?$AAt?$AAi?$AAv?$AAe@ 0001e0f8     MainFrm.obj
 0002:00001178       ??_C@_1GO@PHLPLODI@?$AAD?$AAi?$AAs?$AAc?$AAo?$AAn?$AAn?$AAe?$AAc?$AAt?$AAC?$AAo?$AAd?$AAe?$AA?5?$AAi?$AAg?$AAn?$AAo?$AAr?$AAe?$AAd?$AA?5?$AAb?$AAc?$AAo?$AAs?$AA?5?$AAm?$AA_?$AAd?$AAw@ 0001e178     MainFrm.obj
 0002:000011e8       ??_C@_1FO@HMOAMADL@?$AAD?$AAi?$AAs?$AAc?$AAo?$AAn?$AAn?$AAe?$AAc?$AAt?$AAC?$AAo?$AAd?$AAe?$AA?5?$AAi?$AAg?$AAn?$AAo?$AAr?$AAe?$AAd?$AA?5?$AAb?$AAc?$AAo?$AAs?$AA?5?$AAC?$AAa?$AAl?$AAl@ 0001e1e8     MainFrm.obj
 0002:00001248       ??_C@_1GI@BCFBJPAC@?$AAW?$AAP?$AAS?$AA?5?$AAn?$AAo?$AAt?$AAi?$AAf?$AAi?$AAc?$AAa?$AAt?$AAi?$AAo?$AAn?$AA?5?$AAb?$AAu?$AAb?$AAb?$AAl?$AAe?$AA?5?$AAR?$AAE?$AAM?$AAO?$AAV?$AAE?$AAD?$AA?5@ 0001e248     MainFrm.obj
 0002:000012b0       ??_C@_1DG@CCKFEHGA@?$AAI?$AAt?$AA?5?$AAi?$AAs?$AA?5?$AAW?$AAA?$AAP?$AA?5?$AAI?$AAO?$AAT?$AAA?$AA?5?$AAj?$AAu?$AAs?$AAt?$AA?5?$AAA?$AAC?$AAK?$AA?5?$AAi?$AAt?$AA?$AA@ 0001e2b0     MainFrm.obj
 0002:000012e8       ??_C@_1BG@MAJEEGIE@?$AAI?$AAO?$AAT?$AAA?$AA_?$AAB?$AAE?$AAG?$AAI?$AAN?$AA?$AA@ 0001e2e8     MainFrm.obj
 0002:00001300       ??_C@_1BC@OHNJMDNM@?$AAI?$AAO?$AAT?$AAA?$AA_?$AAE?$AAN?$AAD?$AA?$AA@ 0001e300     MainFrm.obj
 0002:00001314       ??_C@_1BO@OOLLGKIG@?$AAI?$AAT?$AAO?$AAA?$AA_?$AAB?$AAE?$AAG?$AAI?$AAN?$AA_?$AAA?$AAC?$AAK?$AA?$AA@ 0001e314     MainFrm.obj
 0002:00001334       ??_C@_1CA@NDNGFIJB@?$AAI?$AAT?$AAO?$AAA?$AA_?$AAB?$AAE?$AAG?$AAI?$AAN?$AA_?$AAN?$AAA?$AAC?$AAK?$AA?$AA@ 0001e334     MainFrm.obj
 0002:00001354       ??_C@_1BE@ELOIOKNB@?$AAI?$AAO?$AAT?$AAA?$AA_?$AAD?$AAI?$AAA?$AAL?$AA?$AA@ 0001e354     MainFrm.obj
 0002:00001368       ??_C@_1BM@LJOIKJDC@?$AAI?$AAO?$AAT?$AAA?$AA_?$AA1?$AA0?$AA1?$AA2?$AA_?$AAE?$AAR?$AAR?$AA?$AA@ 0001e368     MainFrm.obj
 0002:00001384       ??_C@_1CC@MDIGENCA@?$AAP?$AAH?$AAO?$AAN?$AAE?$AAU?$AAT?$AAI?$AAL?$AAS?$AA_?$AAB?$AAE?$AAG?$AAI?$AAN?$AA?$AA@ 0001e384     MainFrm.obj
 0002:000013a8       ??_C@_1BO@MBMFFGCA@?$AAP?$AAH?$AAO?$AAN?$AAE?$AAU?$AAT?$AAI?$AAL?$AAS?$AA_?$AAE?$AAN?$AAD?$AA?$AA@ 0001e3a8     MainFrm.obj
 0002:000013c8       ??_C@_1CK@NCAHKLGJ@?$AAP?$AAH?$AAO?$AAN?$AAE?$AAU?$AAT?$AAI?$AAL?$AAS?$AA_?$AAB?$AAE?$AAG?$AAI?$AAN?$AA_?$AAA?$AAC?$AAK?$AA?$AA@ 0001e3c8     MainFrm.obj
 0002:000013f4       ??_C@_1CM@OGFDHJCI@?$AAP?$AAH?$AAO?$AAN?$AAE?$AAU?$AAT?$AAI?$AAL?$AAS?$AA_?$AAB?$AAE?$AAG?$AAI?$AAN?$AA_?$AAN?$AAA?$AAC?$AAK?$AA?$AA@ 0001e3f4     MainFrm.obj
 0002:00001420       ??_C@_1CA@FFKJKCCB@?$AAP?$AAH?$AAO?$AAN?$AAE?$AAU?$AAT?$AAI?$AAL?$AAS?$AA_?$AAE?$AAX?$AAI?$AAT?$AA?$AA@ 0001e420     MainFrm.obj
 0002:00001440       ??_C@_1BC@FNALODJM@?$AAA?$AAW?$AA_?$AAB?$AAE?$AAG?$AAI?$AAN?$AA?$AA@ 0001e440     MainFrm.obj
 0002:00001454       ??_C@_1O@LCFHJGAG@?$AAA?$AAW?$AA_?$AAE?$AAN?$AAD?$AA?$AA@ 0001e454     MainFrm.obj
 0002:00001464       ??_C@_1BK@IINCFOMF@?$AAA?$AAW?$AA_?$AAB?$AAE?$AAG?$AAI?$AAN?$AA_?$AAA?$AAC?$AAK?$AA?$AA@ 0001e464     MainFrm.obj
 0002:00001480       ??_C@_1BM@CJDGNGIL@?$AAA?$AAW?$AA_?$AAB?$AAE?$AAG?$AAI?$AAN?$AA_?$AAN?$AAA?$AAC?$AAK?$AA?$AA@ 0001e480     MainFrm.obj
 0002:0000149c       ??_C@_1BA@NBDJACH@?$AAA?$AAW?$AA_?$AAE?$AAX?$AAI?$AAT?$AA?$AA@ 0001e49c     MainFrm.obj
 0002:000014ac       ??_C@_1BM@NNDEDBAN@?$AAU?$AAP?$AAD?$AAA?$AAT?$AAE?$AAR?$AA_?$AAB?$AAE?$AAG?$AAI?$AAN?$AA?$AA@ 0001e4ac     MainFrm.obj
 0002:000014c8       ??_C@_1BI@KBKNMDLB@?$AAU?$AAP?$AAD?$AAA?$AAT?$AAE?$AAR?$AA_?$AAE?$AAN?$AAD?$AA?$AA@ 0001e4c8     MainFrm.obj
 0002:000014e0       ??_C@_1CE@BDGOPNCM@?$AAU?$AAP?$AAD?$AAA?$AAT?$AAE?$AAR?$AA_?$AAB?$AAE?$AAG?$AAI?$AAN?$AA_?$AAA?$AAC?$AAK?$AA?$AA@ 0001e4e0     MainFrm.obj
 0002:00001504       ??_C@_1CG@OJFFPHMA@?$AAU?$AAP?$AAD?$AAA?$AAT?$AAE?$AAR?$AA_?$AAB?$AAE?$AAG?$AAI?$AAN?$AA_?$AAN?$AAA?$AAC?$AAK?$AA?$AA@ 0001e504     MainFrm.obj
 0002:0000152c       ??_C@_1CA@GHJNFPHB@?$AAU?$AAP?$AAD?$AAA?$AAT?$AAE?$AAR?$AA_?$AAE?$AAN?$AAD?$AA_?$AAA?$AAC?$AAK?$AA?$AA@ 0001e52c     MainFrm.obj
 0002:0000154c       ??_C@_1CC@NOJIGCOO@?$AAU?$AAP?$AAD?$AAA?$AAT?$AAE?$AAR?$AA_?$AAE?$AAN?$AAD?$AA_?$AAN?$AAA?$AAC?$AAK?$AA?$AA@ 0001e54c     MainFrm.obj
 0002:00001570       ??_7CMipErrorDlg@@6B@      0001e570     miperrdlg.obj
 0002:00001574       ??_C@_1BG@EOKOAFMK@?$AA?$CI?$AAE?$AAr?$AAr?$AAo?$AAr?$AA?5?$AA?$CF?$AAd?$AA?$CJ?$AA?$AA@ 0001e574     miperrdlg.obj
 0002:0000158c       ??_C@_1BK@LPEBGBPE@?$AAM?$AAI?$AAP?$AA?5?$AAE?$AAr?$AAr?$AAo?$AAr?$AA?5?$AA?$CF?$AAd?$AA?$AA@ 0001e58c     miperrdlg.obj
 0002:000015a8       ??_7CResultListElement@@6B@ 0001e5a8     resultelement.obj
 0002:000015ac       ??_C@_1BA@CLKPCLJO@?$AAU?$AAP?$AAD?$AAA?$AAT?$AAE?$AAR?$AA?$AA@ 0001e5ac     Session.obj
 0002:000015bc       ??_C@_15NMODLAIO@?$AAA?$AAW?$AA?$AA@ 0001e5bc     Session.obj
 0002:000015c4       ??_C@_1BG@BENLIEFL@?$AAP?$AAh?$AAo?$AAn?$AAe?$AAU?$AAt?$AAi?$AAl?$AAs?$AA?$AA@ 0001e5c4     Session.obj
 0002:000015dc       ??_C@_19DKNABOBL@?$AAI?$AAO?$AAT?$AAA?$AA?$AA@ 0001e5dc     Session.obj
 0002:000015e8       ??_7CSession@@6B@          0001e5e8     Session.obj
 0002:000016a8       ??_C@_1GM@DCLOECDA@?$AAC?$AAS?$AAe?$AAs?$AAs?$AAi?$AAo?$AAn?$AAM?$AAa?$AAn?$AAa?$AAg?$AAe?$AAr?$AA?3?$AA?3?$AAC?$AAh?$AAe?$AAc?$AAk?$AA?5?$AA?$CI?$AA?$CF?$AAd?$AA?$CJ?$AA?5?$AAr?$AAe?$AAt?$AAu@ 0001e6a8     SessionManager.obj
 0002:00001714       ??_C@_1CK@GJDPIPOM@?$AA?4?$AA?2?$AAs?$AAe?$AAs?$AAs?$AAi?$AAo?$AAn?$AAm?$AAa?$AAn?$AAa?$AAg?$AAe?$AAr?$AA?4?$AAc?$AAp?$AAp?$AA?$AA@ 0001e714     SessionManager.obj
 0002:00001740       ??_C@_1EK@DEPPCCNP@?$AAU?$AAp?$AAd?$AAa?$AAt?$AAe?$AAr?$AA?5?$AAo?$AAr?$AAd?$AAe?$AAr?$AAs?$AA?5?$AAP?$AAh?$AAo?$AAn?$AAe?$AA?5?$AAu?$AAt?$AAi?$AAl?$AAi?$AAt?$AAy?$AA?5?$AAt?$AAo?$AA?5@ 0001e740     SessionManager.obj
 0002:000017c0       ??_7CSessionManager@@6B@   0001e7c0     SessionManager.obj
 0002:00001838       ??_C@_0BB@MOGOBHAF@list?$DMT?$DO?5too?5long?$AA@ 0001e838     SessionManager.obj
 0002:000018c0       ??_C@_1GA@CBCEEEJC@?$AAC?$AAr?$AAe?$AAa?$AAt?$AAe?$AA?5?$AAS?$AAe?$AAs?$AAs?$AAi?$AAo?$AAn?$AA?5?$AAf?$AAo?$AAr?$AA?5?$AA?$CF?$AAs?$AA?5?$AAf?$AAa?$AAi?$AAl?$AAe?$AAd?$AA?4?$AA?5?$AAN?$AAo@ 0001e8c0     SessionManager.obj
 0002:00001920       ??_7CStateMachineMgr@@6B@  0001e920     StateMachineMgr.obj
 0002:00001924       ??_C@_1CI@MLEEJICB@?$AAK?$AAi?$AAl?$AAl?$AAA?$AAc?$AAt?$AAi?$AAv?$AAe?$AAS?$AAy?$AAn?$AAc?$AA4?$AAI?$AAO?$AAT?$AAA?$AA?$AA@ 0001e924     StateMachineMgr.obj
 0002:0000194c       ??_C@_1CO@POMBJCLO@?$AAP?$AAh?$AAo?$AAn?$AAe?$AA?5?$AAi?$AAs?$AA?5?$AAn?$AAo?$AAt?$AA?5?$AAa?$AAc?$AAt?$AAi?$AAv?$AAa?$AAt?$AAe?$AAd?$AA?$AA@ 0001e94c     StateMachineMgr.obj
 0002:0000197c       ??_C@_1CO@OJFKALKA@?$AAC?$AAa?$AAn?$AAn?$AAo?$AAt?$AA?5?$AAk?$AAi?$AAl?$AAl?$AA?5?$AAA?$AAc?$AAt?$AAi?$AAv?$AAe?$AAS?$AAy?$AAn?$AAc?$AA?$AA@ 0001e97c     StateMachineMgr.obj
 0002:000019ac       ??_C@_1BA@JKDDHIHE@?$AAR?$AAe?$AAp?$AAl?$AAL?$AAo?$AAg?$AA?$AA@ 0001e9ac     StateMachineMgr.obj
 0002:000019bc       ??_C@_1CA@LGOLPII@?$AAI?$AAn?$AA?5?$AAT?$AAe?$AAt?$AAh?$AAe?$AAr?$AAe?$AAd?$AAM?$AAo?$AAd?$AAe?$AA?$AA@ 0001e9bc     StateMachineMgr.obj
 0002:000019dc       ??_C@_1DI@NDOJBHKA@?$AAG?$AAe?$AAt?$AAC?$AAa?$AAl?$AAl?$AAS?$AAt?$AAa?$AAt?$AAu?$AAs?$AA?$CI?$AA?$CJ?$AA?3?$AA?5?$AAV?$AAO?$AAI?$AAC?$AAE?$AA_?$AAC?$AAA?$AAL?$AAL?$AA?$AA@ 0001e9dc     StateMachineMgr.obj
 0002:00001a18       ??_C@_1EC@NDMKODNN@?$AAG?$AAe?$AAt?$AAC?$AAa?$AAl?$AAl?$AAS?$AAt?$AAa?$AAt?$AAu?$AAs?$AA?$CI?$AA?$CJ?$AA?3?$AA?5?$AAV?$AAO?$AAI?$AAC?$AAE?$AA_?$AAD?$AAA?$AAT?$AAA?$AA_?$AAC?$AAA?$AAL?$AAL@ 0001ea18     StateMachineMgr.obj
 0002:00001a60       ??_C@_1HC@MKACAMKD@?$AAI?$AAn?$AA?5?$AAa?$AAn?$AA?5?$AAa?$AAc?$AAt?$AAi?$AAv?$AAe?$AA?5?$AAD?$AAa?$AAt?$AAa?$AA?5?$AAc?$AAa?$AAl?$AAl?$AA?5?$AA?0?$AA?5?$AAU?$AAn?$AAa?$AAb?$AAl?$AAe?$AA?5@ 0001ea60     StateMachineMgr.obj
 0002:00001ad8       ??_C@_1KA@DAAFLMMG@?$AAU?$AAn?$AAa?$AAb?$AAl?$AAe?$AA?5?$AAt?$AAo?$AA?5?$AAD?$AAi?$AAs?$AAc?$AAo?$AAn?$AAn?$AAe?$AAc?$AAt?$AA?5?$AAt?$AAh?$AAe?$AA?5?$AAu?$AAs?$AAe?$AAr?$AA?5?$AAD?$AAa@ 0001ead8     StateMachineMgr.obj
 0002:00001b78       ??_C@_1CM@MECAIAHA@?$AA?4?$AA?2?$AAs?$AAt?$AAa?$AAt?$AAe?$AAm?$AAa?$AAc?$AAh?$AAi?$AAn?$AAe?$AAm?$AAg?$AAr?$AA?4?$AAc?$AAp?$AAp?$AA?$AA@ 0001eb78     StateMachineMgr.obj
 0002:00001ba4       ??_C@_1DI@GFBBFND@?$AAP?$AAh?$AAo?$AAn?$AAe?$AA?5?$AAi?$AAs?$AA?5?$AAo?$AAf?$AAf?$AA?0?$AAc?$AAa?$AAn?$AA?8?$AAt?$AA?5?$AAs?$AAt?$AAa?$AAr?$AAt?$AA?5?$AA?$CF?$AAs?$AA?$AA@ 0001eba4     StateMachineMgr.obj
 0002:00001bdc       ??_C@_1BC@PCHKAMBP@?$AAP?$AAO?$AAW?$AAE?$AAR?$AA_?$AAO?$AAN?$AA?$AA@ 0001ebdc     StdAfx.obj
 0002:00001bf0       ??_C@_1BE@JGMADFED@?$AAP?$AAO?$AAW?$AAE?$AAR?$AA_?$AAO?$AAF?$AAF?$AA?$AA@ 0001ebf0     StdAfx.obj
 0002:00001c04       ??_C@_1BK@LHMHCDIP@?$AAI?$AAT?$AAO?$AAA?$AA_?$AAE?$AAN?$AAD?$AA_?$AAA?$AAC?$AAK?$AA?$AA@ 0001ec04     StdAfx.obj
 0002:00001c20       ??_C@_1CG@NGJLINHO@?$AAI?$AAO?$AAT?$AAA?$AA_?$AAA?$AAL?$AAI?$AAV?$AAE?$AA_?$AAM?$AAE?$AAS?$AAS?$AAA?$AAG?$AAE?$AA?$AA@ 0001ec20     StdAfx.obj
 0002:00001c48       ??_C@_1CE@JLPOCCBE@?$AAI?$AAO?$AAT?$AAA?$AA_?$AAP?$AAI?$AAN?$AAG?$AA_?$AAM?$AAE?$AAS?$AAS?$AAA?$AAG?$AAE?$AA?$AA@ 0001ec48     StdAfx.obj
 0002:00001c6c       ??_C@_1BM@NCKPFMMC@?$AAI?$AAO?$AAT?$AAA?$AA_?$AAP?$AAI?$AAN?$AAG?$AA_?$AAA?$AAC?$AAK?$AA?$AA@ 0001ec6c     StdAfx.obj
 0002:00001c88       ??_C@_1CI@HGBOCMNH@?$AAI?$AAO?$AAT?$AAA?$AA_?$AAC?$AAR?$AAI?$AAT?$AAI?$AAC?$AAA?$AAL?$AA_?$AAE?$AAR?$AAR?$AAO?$AAR?$AA?$AA@ 0001ec88     StdAfx.obj
 0002:00001cb0       ??_C@_1DA@BHPKMPLG@?$AAI?$AAO?$AAT?$AAA?$AA_?$AAN?$AAO?$AAN?$AA_?$AAC?$AAR?$AAI?$AAT?$AAI?$AAC?$AAA?$AAL?$AA_?$AAE?$AAR?$AAR?$AAO?$AAR?$AA?$AA@ 0001ecb0     StdAfx.obj
 0002:00001ce0       ??_C@_1CC@MLMAKKOO@?$AAK?$AAI?$AAL?$AAL?$AA_?$AAI?$AAO?$AAT?$AAA?$AA_?$AAP?$AAL?$AAE?$AAA?$AAS?$AAE?$AA?$AA@ 0001ece0     StdAfx.obj
 0002:00001d04       ??_C@_1CG@PGHILCBC@?$AAI?$AAO?$AAT?$AAA?$AA_?$AAU?$AAP?$AAD?$AAA?$AAT?$AAE?$AA_?$AAS?$AAT?$AAA?$AAT?$AAU?$AAS?$AA?$AA@ 0001ed04     StdAfx.obj
 0002:00001d2c       ??_C@_1CK@LDMADEEM@?$AAI?$AAO?$AAT?$AAA?$AA_?$AAD?$AAa?$AAt?$AAa?$AA_?$AAP?$AAo?$AAr?$AAt?$AA_?$AAI?$AAn?$AAU?$AAs?$AAe?$AA?$AA@ 0001ed2c     StdAfx.obj
 0002:00001d58       ??_C@_1CO@GLHJIBOI@?$AAI?$AAO?$AAT?$AAA?$AA_?$AAP?$AAR?$AAO?$AAV?$AAI?$AAS?$AAI?$AAO?$AAN?$AAI?$AAN?$AAG?$AA_?$AAD?$AAO?$AAN?$AAE?$AA?$AA@ 0001ed58     StdAfx.obj
 0002:00001d88       ??_C@_1CI@PIELHBKD@?$AAP?$AAH?$AAO?$AAN?$AAE?$AAU?$AAT?$AAI?$AAL?$AAS?$AA_?$AAE?$AAN?$AAD?$AA_?$AAN?$AAA?$AAC?$AAK?$AA?$AA@ 0001ed88     StdAfx.obj
 0002:00001db0       ??_C@_1DC@KNIKGFIB@?$AAP?$AAH?$AAO?$AAN?$AAE?$AAU?$AAT?$AAI?$AAL?$AAS?$AA_?$AAA?$AAL?$AAI?$AAV?$AAE?$AA_?$AAM?$AAE?$AAS?$AAS?$AAA?$AAG?$AAE?$AA?$AA@ 0001edb0     StdAfx.obj
 0002:00001de4       ??_C@_1DA@FCENJAPE@?$AAP?$AAH?$AAO?$AAN?$AAE?$AAU?$AAT?$AAI?$AAL?$AAS?$AA_?$AAP?$AAI?$AAN?$AAG?$AA_?$AAM?$AAE?$AAS?$AAS?$AAA?$AAG?$AAE?$AA?$AA@ 0001ede4     StdAfx.obj
 0002:00001e14       ??_C@_1CI@NPKEBPGG@?$AAP?$AAH?$AAO?$AAN?$AAE?$AAU?$AAT?$AAI?$AAL?$AAS?$AA_?$AAP?$AAI?$AAN?$AAG?$AA_?$AAA?$AAC?$AAK?$AA?$AA@ 0001ee14     StdAfx.obj
 0002:00001e3c       ??_C@_1BG@FJAKJBPC@?$AAA?$AAW?$AA_?$AAE?$AAN?$AAD?$AA_?$AAA?$AAC?$AAK?$AA?$AA@ 0001ee3c     StdAfx.obj
 0002:00001e54       ??_C@_1CC@FGHONIMK@?$AAA?$AAW?$AA_?$AAA?$AAL?$AAI?$AAV?$AAE?$AA_?$AAM?$AAE?$AAS?$AAS?$AAA?$AAG?$AAE?$AA?$AA@ 0001ee54     StdAfx.obj
 0002:00001e78       ??_C@_1CA@MMOGHMIB@?$AAA?$AAW?$AA_?$AAP?$AAI?$AAN?$AAG?$AA_?$AAM?$AAE?$AAS?$AAS?$AAA?$AAG?$AAE?$AA?$AA@ 0001ee78     StdAfx.obj
 0002:00001e98       ??_C@_1BI@JFAFBGID@?$AAA?$AAW?$AA_?$AAP?$AAI?$AAN?$AAG?$AA_?$AAA?$AAC?$AAK?$AA?$AA@ 0001ee98     StdAfx.obj
 0002:00001eb0       ??_C@_1CG@POBHOMMK@?$AAR?$AAI?$AAL?$AA_?$AAS?$AAT?$AAA?$AAT?$AAU?$AAS?$AA_?$AAC?$AAH?$AAA?$AAN?$AAG?$AAE?$AAD?$AA?$AA@ 0001eeb0     StdAfx.obj
 0002:00001ed8       ??_C@_1BO@NKICKCPO@?$AAR?$AAI?$AAL?$AA_?$AAD?$AAB?$AAG?$AA_?$AAN?$AAO?$AAT?$AAI?$AAF?$AAY?$AA?$AA@ 0001eed8     StdAfx.obj
 0002:00001ef8       ??_C@_1CG@HIPGCNFB@?$AAR?$AAI?$AAL?$AA_?$AAT?$AAE?$AAC?$AAH?$AAH?$AAD?$AAR?$AA_?$AAN?$AAO?$AAT?$AAI?$AAF?$AAY?$AA?$AA@ 0001eef8     StdAfx.obj
 0002:00001f20       ??_C@_1DA@MPHILDIE@?$AAR?$AAI?$AAL?$AA_?$AAI?$AAO?$AAT?$AAA?$AA_?$AAS?$AAT?$AAA?$AAT?$AAU?$AAS?$AA_?$AAC?$AAH?$AAA?$AAN?$AAG?$AAE?$AAD?$AA?$AA@ 0001ef20     StdAfx.obj
 0002:00001f50       ??_C@_1CC@BEOCDLIL@?$AAR?$AAI?$AAL?$AA_?$AAI?$AAO?$AAT?$AAA?$AA_?$AAW?$AAA?$AAP?$AA_?$AAU?$AAR?$AAI?$AA?$AA@ 0001ef50     StdAfx.obj
 0002:00001f74       ??_C@_1CC@POEPKLA@?$AAR?$AAI?$AAL?$AA_?$AAP?$AAD?$AAS?$AAM?$AA_?$AAP?$AAD?$AA_?$AAD?$AAA?$AAT?$AAA?$AA?$AA@ 0001ef74     StdAfx.obj
 0002:00001f98       ??_C@_1CC@DHEBFOCI@?$AAR?$AAI?$AAL?$AA_?$AAP?$AAD?$AAS?$AAM?$AA_?$AAP?$AAD?$AA_?$AAD?$AAO?$AAN?$AAE?$AA?$AA@ 0001ef98     StdAfx.obj
 0002:00001fbc       ??_C@_1CA@IJMMNJBM@?$AAR?$AAI?$AAL?$AA_?$AAP?$AAD?$AAS?$AAM?$AA_?$AAP?$AAD?$AA_?$AAE?$AAN?$AAD?$AA?$AA@ 0001efbc     StdAfx.obj
 0002:00001fdc       ??_C@_1CE@DKNHCEGP@?$AAR?$AAI?$AAL?$AA_?$AAP?$AAD?$AAS?$AAM?$AA_?$AAP?$AAD?$AA_?$AAB?$AAE?$AAG?$AAI?$AAN?$AA?$AA@ 0001efdc     StdAfx.obj
 0002:00002000       ??_C@_1DG@ENNLKGLF@?$AAR?$AAI?$AAL?$AA_?$AAP?$AAD?$AAS?$AAM?$AA_?$AAP?$AAD?$AA_?$AAU?$AAP?$AAD?$AAA?$AAT?$AAE?$AA_?$AAF?$AAA?$AAI?$AAL?$AAU?$AAR?$AAE?$AA?$AA@ 0001f000     StdAfx.obj
 0002:00002038       ??_C@_1CK@FFHNCNLC@?$AAR?$AAI?$AAL?$AA_?$AAP?$AAD?$AAS?$AAM?$AA_?$AAP?$AAD?$AA_?$AAD?$AAL?$AAD?$AA_?$AAD?$AAA?$AAT?$AAA?$AA?$AA@ 0001f038     StdAfx.obj
 0002:00002064       ??_C@_1CK@GNNIIJCK@?$AAR?$AAI?$AAL?$AA_?$AAP?$AAD?$AAS?$AAM?$AA_?$AAP?$AAD?$AA_?$AAD?$AAL?$AAD?$AA_?$AAD?$AAO?$AAN?$AAE?$AA?$AA@ 0001f064     StdAfx.obj
 0002:00002090       ??_C@_1CI@IINDIONI@?$AAR?$AAI?$AAL?$AA_?$AAP?$AAD?$AAS?$AAM?$AA_?$AAP?$AAD?$AA_?$AAD?$AAL?$AAD?$AA_?$AAE?$AAN?$AAD?$AA?$AA@ 0001f090     StdAfx.obj
 0002:000020b8       ??_C@_1CM@BAFGFLAD@?$AAR?$AAI?$AAL?$AA_?$AAP?$AAD?$AAS?$AAM?$AA_?$AAP?$AAD?$AA_?$AAD?$AAL?$AAD?$AA_?$AAB?$AAE?$AAG?$AAI?$AAN?$AA?$AA@ 0001f0b8     StdAfx.obj
 0002:000020e4       ??_C@_1CE@GDPLDIKM@?$AAR?$AAI?$AAL?$AA_?$AAP?$AAD?$AAS?$AAM?$AA_?$AAP?$AAA?$AA_?$AAP?$AAA?$AAR?$AAA?$AAM?$AA?$AA@ 0001f0e4     StdAfx.obj
 0002:00002108       ??_C@_1CE@ILHCKNGC@?$AAR?$AAI?$AAL?$AA_?$AAC?$AAA?$AAL?$AAL?$AA_?$AAB?$AAY?$AAT?$AAE?$AA_?$AAC?$AAT?$AAR?$AA?$AA@ 0001f108     StdAfx.obj
 0002:0000212c       ??_7CUSSDDialog@@6B@       0001f12c     USSDDialog.obj
 0002:00002130       ??_C@_1CC@BHNILJJG@?$AA?4?$AA?2?$AAU?$AAS?$AAS?$AAD?$AAD?$AAi?$AAa?$AAl?$AAo?$AAg?$AA?4?$AAc?$AAp?$AAp?$AA?$AA@ 0001f130     USSDDialog.obj
 0002:00002158       ??_C@_1EC@JOGNAECE@?$AAC?$AAr?$AAe?$AAa?$AAt?$AAe?$AA?5?$AAd?$AAi?$AAa?$AAl?$AAo?$AAg?$AA?5?$AAf?$AAa?$AAi?$AAl?$AAe?$AAd?$AA?0?$AA?5?$AAe?$AAr?$AAr?$AAo?$AAr?$AA?5?$AA?$DN?$AA?5?$AA?$CF?$AAd@ 0001f158     USSDDialog.obj
 0002:0000219c       ??_C@_1O@JDLOHAN@?$AAD?$AAe?$AAl?$AAe?$AAt?$AAe?$AA?$AA@ 0001f19c     winmodemstat.obj
 0002:000021ac       ??_C@_1BC@GCKHIPE@?$AAN?$AAo?$AAR?$AAe?$AAm?$AAo?$AAv?$AAe?$AA?$AA@ 0001f1ac     winmodemstat.obj
 0002:000021c0       ??_C@_1BI@JFAIJMHL@?$AAF?$AAo?$AAr?$AAc?$AAe?$AAR?$AAe?$AAm?$AAo?$AAv?$AAe?$AA?$AA@ 0001f1c0     winmodemstat.obj
 0002:000021d8       ??_C@_17LLMMEOJD@?$AAV?$AAa?$AAl?$AA?$AA@ 0001f1d8     winmodemstat.obj
 0002:000021e0       ??_C@_13OPKGLAFF@?$AAB?$AA?$AA@ 0001f1e0     winmodemstat.obj
 0002:000021e4       ??_C@_13MKMNOPIJ@?$AAD?$AA?$AA@ 0001f1e4     winmodemstat.obj
 0002:000021e8       ??_C@_13LHMFKAAD@?$AAM?$AA?$AA@ 0001f1e8     winmodemstat.obj
 0002:000021ec       ??_C@_13HADIAKP@?$AAS?$AA?$AA@ 0001f1ec     winmodemstat.obj
 0002:00002210       ??_7CModemStatus@@6B@      0001f210     winmodemstat.obj
 0002:00002214       ??_C@_1CG@IOFFODIG@?$AAM?$AAO?$AAD?$AAE?$AAM?$AA_?$AAO?$AAN?$AA_?$AAO?$AAF?$AAF?$AA_?$AAE?$AAV?$AAE?$AAN?$AAT?$AA?$AA@ 0001f214     winmodemstat.obj
 0002:00002240       ??_C@_1FO@BDBEHFFH@?$AA?4?$AA?4?$AA?2?$AA?4?$AA?4?$AA?2?$AA?4?$AA?4?$AA?2?$AAR?$AAI?$AAL?$AAD?$AAr?$AAi?$AAv?$AAe?$AAr?$AA?2?$AAC?$AAo?$AAm?$AAm?$AAo?$AAn?$AA?2?$AAs?$AAr?$AAc?$AA?2?$AAw?$AAi@ 0001f240     winmodemstat.obj
 0002:000022a0       ??_C@_1JO@DKICHNLH@?$AAS?$AAe?$AAn?$AAd?$AA?5?$AAm?$AAe?$AAs?$AAs?$AAa?$AAg?$AAe?$AA?5?$AAt?$AAi?$AAm?$AAe?$AAo?$AAu?$AAt?$AA?5?$AAf?$AAr?$AAo?$AAm?$AA?5?$AAw?$AAi?$AAn?$AAm?$AAo?$AAd@ 0001f2a0     winmodemstat.obj
 0002:00002340       ??_C@_1GG@MLOAOBHO@?$AAU?$AAp?$AAd?$AAa?$AAt?$AAe?$AAC?$AAa?$AAl?$AAl?$AAT?$AAy?$AAp?$AAe?$AAA?$AAn?$AAd?$AAS?$AAt?$AAa?$AAt?$AAu?$AAs?$AA?5?$AAc?$AAa?$AAn?$AAn?$AAo?$AAt?$AA?5?$AAh@ 0001f340     winmodemstat.obj
 0002:000023a8       ??_C@_1JG@JMBAMLCB@?$AAI?$AAn?$AAv?$AAa?$AAl?$AAi?$AAd?$AA?5?$AAs?$AAt?$AAa?$AAt?$AAe?$AA?3?$AA?5?$AAm?$AA_?$AAC?$AAa?$AAl?$AAl?$AAT?$AAy?$AAp?$AAe?$AA?5?$AA?$DN?$AA?5?$AA?$CF?$AAd?$AA?5?$AAb@ 0001f3a8     winmodemstat.obj
 0002:00002440       ??_C@_1FO@GFODOKOF@?$AAI?$AAn?$AAv?$AAa?$AAl?$AAi?$AAd?$AA?5?$AAs?$AAt?$AAa?$AAt?$AAe?$AA?3?$AA?5?$AAm?$AA_?$AAC?$AAa?$AAl?$AAl?$AAT?$AAy?$AAp?$AAe?$AA?5?$AA?$DN?$AA?5?$AA?$CF?$AAd?$AA?5?$AAb@ 0001f440     winmodemstat.obj
 0002:000024a0       ??_C@_1DK@CMAHCKEF@?$AAI?$AAn?$AAv?$AAa?$AAl?$AAi?$AAd?$AA?5?$AAc?$AAa?$AAl?$AAl?$AAE?$AAv?$AAe?$AAn?$AAt?$AAM?$AAa?$AAs?$AAk?$AA?5?$AA?$DN?$AA?5?$AA0?$AAx?$AA?$CF?$AAx?$AA?$AA@ 0001f4a0     winmodemstat.obj
 0002:000024dc       ??_C@_1CI@CHFKALHP@?$AAU?$AAN?$AAC?$AAH?$AAG?$AA?0?$AA?5?$AAi?$AAn?$AAv?$AAa?$AAl?$AAi?$AAd?$AA?5?$AAc?$AAa?$AAs?$AAe?$AA?$AA@ 0001f4dc     winmodemstat.obj
 0002:00002508       ??_C@_1GA@COEPBEFB@?$AAW?$AAr?$AAo?$AAn?$AAg?$AA?5?$AAp?$AAa?$AAr?$AAa?$AAm?$AA?5?$AAf?$AAo?$AAr?$AA?5?$AAG?$AAe?$AAt?$AAD?$AAe?$AAt?$AAa?$AAi?$AAl?$AAE?$AAr?$AAr?$AAo?$AAr?$AAC?$AAo@ 0001f508     winmodemstat.obj
 0002:00002638       ??_C@_1NK@HKFOPGPM@?$AAI?$AAn?$AAv?$AAa?$AAl?$AAi?$AAd?$AA?5?$AAu?$AAs?$AAe?$AA?5?$AAo?$AAf?$AA?5?$AAA?$AAd?$AAd?$AAR?$AAe?$AAs?$AAu?$AAl?$AAt?$AAI?$AAt?$AAe?$AAm?$AA?5?$AAo?$AAn?$AA?5@ 0001f638     winmodemstat.obj
 0002:00002780       ??_C@_1GE@NCBFCKEM@?$AAA?$AAb?$AAo?$AAu?$AAt?$AA?5?$AAt?$AAo?$AA?5?$AAc?$AAa?$AAl?$AAl?$AA?5?$AAT?$AAe?$AAr?$AAm?$AAi?$AAn?$AAa?$AAt?$AAe?$AAP?$AAr?$AAo?$AAc?$AAe?$AAs?$AAs?$AA?5?$AAi@ 0001f780     winmodemstat.obj
 0002:000027e8       ??_C@_1FC@IDFJCPGP@?$AAC?$AAA?$AAT?$AAC?$AAH?$AA_?$AAT?$AAH?$AAE?$AA_?$AAE?$AAR?$AAR?$AAO?$AAR?$AA?5?$AAb?$AAu?$AAt?$AA?5?$AAc?$AAa?$AAn?$AAn?$AAo?$AAt?$AA?5?$AAp?$AAo?$AAs?$AAt?$AA?5@ 0001f7e8     winmodemstat.obj
 0002:00002918       ??_C@_1FO@HEAAPBIE@?$AAC?$AAa?$AAr?$AAr?$AAi?$AAe?$AAr?$AA?5?$AAI?$AAn?$AAd?$AAe?$AAx?$AA?5?$AAC?$AAh?$AAn?$AAa?$AAg?$AAe?$AAd?$AA?5?$AAN?$AAO?$AAT?$AAI?$AAF?$AAY?$AA_?$AAC?$AAA?$AAR@ 0001f918     winmodemstat.obj
 0002:00002978       ??_C@_1DK@FPIKNIHL@?$AAR?$AAI?$AAL?$AA_?$AAN?$AAO?$AAT?$AAI?$AAF?$AAY?$AA_?$AAP?$AAD?$AAP?$AA_?$AAI?$AAN?$AAA?$AAC?$AAT?$AA_?$AAF?$AAA?$AAI?$AAL?$AA_?$AAE?$AA?5?$AA?$AA@ 0001f978     winmodemstat.obj
 0002:000029b8       ??_C@_1KE@BGFKGAIL@?$AAT?$AAe?$AAl?$AAl?$AA?5?$AAo?$AAu?$AAr?$AA?5?$AAa?$AAp?$AAp?$AAs?$AA?5?$AAt?$AAo?$AA?5?$AAc?$AAl?$AAe?$AAa?$AAn?$AA?5?$AAu?$AAp?$AA?5?$AAt?$AAh?$AAe?$AA?5?$AAc?$AAa@ 0001f9b8     winmodemstat.obj
 0002:00002a60       ??_C@_1GA@DMPCLOLH@?$AAR?$AAI?$AAL?$AA_?$AAD?$AAe?$AAv?$AAS?$AAp?$AAe?$AAc?$AAi?$AAf?$AAi?$AAc?$AA?5?$AAf?$AAa?$AAi?$AAl?$AAe?$AAd?$AA?5?$AAr?$AAe?$AAt?$AAu?$AAr?$AAn?$AA?3?$AA?5?$AA?$CF@ 0001fa60     winmodemstat.obj
 0002:00002b30       ??_C@_1GA@JKFDDEPE@?$AAD?$AAo?$AAn?$AA?8?$AAt?$AA?5?$AAk?$AAn?$AAo?$AAw?$AA?5?$AAh?$AAo?$AAw?$AA?5?$AAt?$AAo?$AA?5?$AAA?$AAd?$AAd?$AAR?$AAe?$AAs?$AAu?$AAl?$AAt?$AAI?$AAt?$AAe?$AAm?$AA?5@ 0001fb30     winmodemstat.obj
 0002:00002c00       ??_C@_1EK@PLMMIOKB@?$AAR?$AAI?$AAL?$AA_?$AAI?$AAn?$AAi?$AAt?$AAi?$AAa?$AAl?$AAi?$AAz?$AAe?$AA?5?$AAf?$AAa?$AAi?$AAl?$AAe?$AAd?$AA?5?$AAh?$AAR?$AAe?$AAs?$AAu?$AAl?$AAt?$AA?5?$AA?$DN?$AA?5@ 0001fc00     winmodemstat.obj
 0002:00002c50       ??_7bad_alloc@std@@6B@     0001fc50     libcpmt:string.obj
 0002:00002c5c       ??_7logic_error@std@@6B@   0001fc5c     libcpmt:string.obj
 0002:00002c68       ??_7length_error@std@@6B@  0001fc68     libcpmt:string.obj
 0002:00002c74       ??_7out_of_range@std@@6B@  0001fc74     libcpmt:string.obj
 0002:00002cc8       ??_C@_0BA@JFNIOLAK@string?5too?5long?$AA@ 0001fcc8     libcpmt:string.obj
 0002:00002d24       ??_C@_0BI@CFPLBAOH@invalid?5string?5position?$AA@ 0001fd24     libcpmt:string.obj
 0002:00002d3c       GUID_ATLVer30              0001fd3c     atls:atlbase.obj
 0002:00002d4c       GUID_ATLVer70              0001fd4c     atls:atlbase.obj
 0002:00002d5c       IID_IPersistStream         0001fd5c     uuid:objidl_i_guid12.obj
 0002:00002d6c       ??_R4bad_alloc@std@@6B@    0001fd6c     libcpmt:string.obj
 0002:00002d80       ??_R3bad_alloc@std@@8      0001fd80     libcpmt:string.obj
 0002:00002d90       ??_R2bad_alloc@std@@8      0001fd90     libcpmt:string.obj
 0002:00002d9c       ??_R1A@?0A@EA@bad_alloc@std@@8 0001fd9c     libcpmt:string.obj
 0002:00002db8       ??_R1A@?0A@EA@exception@std@@8 0001fdb8     libcpmt:string.obj
 0002:00002dd4       ??_R3exception@std@@8      0001fdd4     libcpmt:string.obj
 0002:00002de4       ??_R2exception@std@@8      0001fde4     libcpmt:string.obj
 0002:00002dec       ??_R4logic_error@std@@6B@  0001fdec     libcpmt:string.obj
 0002:00002e00       ??_R3logic_error@std@@8    0001fe00     libcpmt:string.obj
 0002:00002e10       ??_R2logic_error@std@@8    0001fe10     libcpmt:string.obj
 0002:00002e1c       ??_R1A@?0A@EA@logic_error@std@@8 0001fe1c     libcpmt:string.obj
 0002:00002e38       ??_R4length_error@std@@6B@ 0001fe38     libcpmt:string.obj
 0002:00002e4c       ??_R3length_error@std@@8   0001fe4c     libcpmt:string.obj
 0002:00002e5c       ??_R2length_error@std@@8   0001fe5c     libcpmt:string.obj
 0002:00002e6c       ??_R1A@?0A@EA@length_error@std@@8 0001fe6c     libcpmt:string.obj
 0002:00002e88       ??_R4out_of_range@std@@6B@ 0001fe88     libcpmt:string.obj
 0002:00002e9c       ??_R3out_of_range@std@@8   0001fe9c     libcpmt:string.obj
 0002:00002eac       ??_R2out_of_range@std@@8   0001feac     libcpmt:string.obj
 0002:00002ebc       ??_R1A@?0A@EA@out_of_range@std@@8 0001febc     libcpmt:string.obj
 0002:00002fb4       _TI2?AVbad_alloc@std@@     0001ffb4     SessionManager.obj
 0002:00002fc4       _CTA2?AVbad_alloc@std@@    0001ffc4     SessionManager.obj
 0002:00002fd0       _CT??_R0?AVbad_alloc@std@@@8??0bad_alloc@std@@QAA@ABV01@@Z12 0001ffd0     SessionManager.obj
 0002:00002fec       _CT??_R0?AVexception@std@@@8??0exception@std@@QAA@ABV01@@Z12 0001ffec     SessionManager.obj
 0002:00003008       _TI3?AVlength_error@std@@  00020008     SessionManager.obj
 0002:00003018       _CTA3?AVlength_error@std@@ 00020018     SessionManager.obj
 0002:00003028       _CT??_R0?AVlength_error@std@@@8??0length_error@std@@QAA@ABV01@@Z40 00020028     SessionManager.obj
 0002:00003044       _CT??_R0?AVlogic_error@std@@@8??0logic_error@std@@QAA@ABV01@@Z40 00020044     SessionManager.obj
 0002:00003060       _TI3?AVout_of_range@std@@  00020060     libcpmt:string.obj
 0002:00003070       _CTA3?AVout_of_range@std@@ 00020070     libcpmt:string.obj
 0002:00003080       _CT??_R0?AVout_of_range@std@@@8??0out_of_range@std@@QAA@ABV01@@Z40 00020080     libcpmt:string.obj
 0002:0000309c       __IMPORT_DESCRIPTOR_sw_utilityG 0002009c     sw_utilityG:sw_utilityG.dll
 0002:000030b0       __IMPORT_DESCRIPTOR_ril    000200b0     ril:ril.dll
 0002:000030c4       __IMPORT_DESCRIPTOR_toolhelp 000200c4     toolhelp:toolhelp.dll
 0002:000030d8       __IMPORT_DESCRIPTOR_COREDLL 000200d8     coredll:COREDLL.dll
 0002:000030ec       __IMPORT_DESCRIPTOR_AYGSHELL 000200ec     aygshell:AYGSHELL.dll
 0002:00003100       __NULL_IMPORT_DESCRIPTOR   00020100     sw_utilityG:sw_utilityG.dll
 0003:00000000       __imp_ExitWindowsEx        00021000     aygshell:AYGSHELL.dll
 0003:00000004       __imp_SHCreateMenuBar      00021004     aygshell:AYGSHELL.dll
 0003:00000008       __imp_SHNotificationAdd    00021008     aygshell:AYGSHELL.dll
 0003:0000000c       __imp_SHNotificationRemove 0002100c     aygshell:AYGSHELL.dll
 0003:00000010       __imp_SHNotificationUpdate 00021010     aygshell:AYGSHELL.dll
 0003:00000014       __imp_SHNotificationGetData 00021014     aygshell:AYGSHELL.dll
 0003:00000018       __imp_SHEnableSoftkey      00021018     aygshell:AYGSHELL.dll
 0003:0000001c       __imp_SHInitDialog         0002101c     aygshell:AYGSHELL.dll
 0003:00000020       \177AYGSHELL_NULL_THUNK_DATA 00021020     aygshell:AYGSHELL.dll
 0003:00000024       __imp_TlsSetValue          00021024     coredll:COREDLL.dll
 0003:00000028       __imp_TlsCall              00021028     coredll:COREDLL.dll
 0003:0000002c       __imp_memmove              0002102c     coredll:COREDLL.dll
 0003:00000030       __imp_?terminate@std@@YAXXZ 00021030     coredll:COREDLL.dll
 0003:00000034       __imp_strcmp               00021034     coredll:COREDLL.dll
 0003:00000038       __imp_TlsGetValue          00021038     coredll:COREDLL.dll
 0003:0000003c       __imp_LocalFree            0002103c     coredll:COREDLL.dll
 0003:00000040       __imp_LocalSize            00021040     coredll:COREDLL.dll
 0003:00000044       __imp_LocalAlloc           00021044     coredll:COREDLL.dll
 0003:00000048       __imp_LocalReAlloc         00021048     coredll:COREDLL.dll
 0003:0000004c       __imp___report_gsfailure   0002104c     coredll:COREDLL.dll
 0003:00000050       __imp__XcptFilter          00021050     coredll:COREDLL.dll
 0003:00000054       __imp_InterlockedCompareExchange 00021054     coredll:COREDLL.dll
 0003:00000058       __imp_GetModuleHandleW     00021058     coredll:COREDLL.dll
 0003:0000005c       __imp_RasGetConnectStatus  0002105c     coredll:COREDLL.dll
 0003:00000060       __imp_FindWindowW          00021060     coredll:COREDLL.dll
 0003:00000064       __imp_??_U@YAPAXI@Z        00021064     coredll:COREDLL.dll
 0003:00000068       __imp___security_gen_cookie 00021068     coredll:COREDLL.dll
 0003:0000006c       __imp_SetWindowLongW       0002106c     coredll:COREDLL.dll
 0003:00000070       __imp_??_V@YAXPAX@Z        00021070     coredll:COREDLL.dll
 0003:00000074       __imp_TerminateProcess     00021074     coredll:COREDLL.dll
 0003:00000078       __imp_free                 00021078     coredll:COREDLL.dll
 0003:0000007c       __imp_SendMessageTimeout   0002107c     coredll:COREDLL.dll
 0003:00000080       __imp___C_specific_handler 00021080     coredll:COREDLL.dll
 0003:00000084       __imp_RaiseException       00021084     coredll:COREDLL.dll
 0003:00000088       __imp_GetDlgItemTextW      00021088     coredll:COREDLL.dll
 0003:0000008c       __imp_Sleep                0002108c     coredll:COREDLL.dll
 0003:00000090       __imp_FindClose            00021090     coredll:COREDLL.dll
 0003:00000094       __imp_FindFirstFileW       00021094     coredll:COREDLL.dll
 0003:00000098       __imp_WaitForSingleObject  00021098     coredll:COREDLL.dll
 0003:0000009c       __imp_wcscpy               0002109c     coredll:COREDLL.dll
 0003:000000a0       __imp_GetLastError         000210a0     coredll:COREDLL.dll
 0003:000000a4       __imp_LoadLibraryW         000210a4     coredll:COREDLL.dll
 0003:000000a8       __imp_CreateMutexW         000210a8     coredll:COREDLL.dll
 0003:000000ac       __imp_GetMessageW          000210ac     coredll:COREDLL.dll
 0003:000000b0       __imp_DispatchMessageW     000210b0     coredll:COREDLL.dll
 0003:000000b4       __imp_TranslateMessage     000210b4     coredll:COREDLL.dll
 0003:000000b8       __imp_wcsrchr              000210b8     coredll:COREDLL.dll
 0003:000000bc       __imp_EventModify          000210bc     coredll:COREDLL.dll
 0003:000000c0       __imp_??3@YAXPAX@Z         000210c0     coredll:COREDLL.dll
 0003:000000c4       __imp_CreateEventW         000210c4     coredll:COREDLL.dll
 0003:000000c8       __imp_InitializeCriticalSection 000210c8     coredll:COREDLL.dll
 0003:000000cc       __imp_??2@YAPAXI@Z         000210cc     coredll:COREDLL.dll
 0003:000000d0       __imp__wcsicmp             000210d0     coredll:COREDLL.dll
 0003:000000d4       __imp_CloseHandle          000210d4     coredll:COREDLL.dll
 0003:000000d8       __imp_DeleteCriticalSection 000210d8     coredll:COREDLL.dll
 0003:000000dc       __imp_LeaveCriticalSection 000210dc     coredll:COREDLL.dll
 0003:000000e0       __imp_EnterCriticalSection 000210e0     coredll:COREDLL.dll
 0003:000000e4       __imp_NKDbgPrintfW         000210e4     coredll:COREDLL.dll
 0003:000000e8       __imp_CreateThread         000210e8     coredll:COREDLL.dll
 0003:000000ec       __imp_MessageBoxW          000210ec     coredll:COREDLL.dll
 0003:000000f0       __imp_LoadStringW          000210f0     coredll:COREDLL.dll
 0003:000000f4       __imp_CreateProcessW       000210f4     coredll:COREDLL.dll
 0003:000000f8       __imp_SystemIdleTimerReset 000210f8     coredll:COREDLL.dll
 0003:000000fc       __imp_PostMessageW         000210fc     coredll:COREDLL.dll
 0003:00000100       __imp_RegisterWindowMessageW 00021100     coredll:COREDLL.dll
 0003:00000104       __imp_SetDlgItemTextW      00021104     coredll:COREDLL.dll
 0003:00000108       __imp_wsprintfW            00021108     coredll:COREDLL.dll
 0003:0000010c       __imp_ShowWindow           0002110c     coredll:COREDLL.dll
 0003:00000110       __imp_SetForegroundWindow  00021110     coredll:COREDLL.dll
 0003:00000114       __imp_memset               00021114     coredll:COREDLL.dll
 0003:00000118       __imp_GetWindowLongW       00021118     coredll:COREDLL.dll
 0003:0000011c       __imp_DestroyWindow        0002111c     coredll:COREDLL.dll
 0003:00000120       __imp_EnableWindow         00021120     coredll:COREDLL.dll
 0003:00000124       __imp_GetDlgItem           00021124     coredll:COREDLL.dll
 0003:00000128       __imp_RasHangUp            00021128     coredll:COREDLL.dll
 0003:0000012c       __imp_CreateDialogIndirectParamW 0002112c     coredll:COREDLL.dll
 0003:00000130       __imp_LoadResource         00021130     coredll:COREDLL.dll
 0003:00000134       __imp_FindResourceW        00021134     coredll:COREDLL.dll
 0003:00000138       __imp_KillTimer            00021138     coredll:COREDLL.dll
 0003:0000013c       __imp_LoadImageW           0002113c     coredll:COREDLL.dll
 0003:00000140       __imp_SetTimer             00021140     coredll:COREDLL.dll
 0003:00000144       __imp_RegCloseKey          00021144     coredll:COREDLL.dll
 0003:00000148       __imp_RegSetValueExW       00021148     coredll:COREDLL.dll
 0003:0000014c       __imp_RegQueryValueExW     0002114c     coredll:COREDLL.dll
 0003:00000150       __imp_RegOpenKeyExW        00021150     coredll:COREDLL.dll
 0003:00000154       __imp_wcscmp               00021154     coredll:COREDLL.dll
 0003:00000158       __imp_wcsncpy              00021158     coredll:COREDLL.dll
 0003:0000015c       __imp_wcslen               0002115c     coredll:COREDLL.dll
 0003:00000160       __imp_RasEnumConnections   00021160     coredll:COREDLL.dll
 0003:00000164       __imp_SetSystemTime        00021164     coredll:COREDLL.dll
 0003:00000168       __imp_memcpy               00021168     coredll:COREDLL.dll
 0003:0000016c       __imp_RegisterClassW       0002116c     coredll:COREDLL.dll
 0003:00000170       __imp_GetStockObject       00021170     coredll:COREDLL.dll
 0003:00000174       __imp_LoadIconW            00021174     coredll:COREDLL.dll
 0003:00000178       __imp_CreateWindowExW      00021178     coredll:COREDLL.dll
 0003:0000017c       __imp_DefWindowProcW       0002117c     coredll:COREDLL.dll
 0003:00000180       __imp_SetWindowTextW       00021180     coredll:COREDLL.dll
 0003:00000184       __imp_BringWindowToTop     00021184     coredll:COREDLL.dll
 0003:00000188       __imp_strlen               00021188     coredll:COREDLL.dll
 0003:0000018c       __imp_??0exception@std@@QAA@PBD@Z 0002118c     coredll:COREDLL.dll
 0003:00000190       __imp_?what@exception@std@@UBAPBDXZ 00021190     coredll:COREDLL.dll
 0003:00000194       __imp_??1exception@std@@UAA@XZ 00021194     coredll:COREDLL.dll
 0003:00000198       __imp___rt_udiv            00021198     coredll:COREDLL.dll
 0003:0000019c       __imp___CxxThrowException  0002119c     coredll:COREDLL.dll
 0003:000001a0       __imp_??_7type_info@@6B@   000211a0     coredll:COREDLL.dll
 0003:000001a4       __imp_??0exception@std@@QAA@ABV01@@Z 000211a4     coredll:COREDLL.dll
 0003:000001a8       __imp_??0exception@std@@QAA@XZ 000211a8     coredll:COREDLL.dll
 0003:000001ac       __imp_wcscat               000211ac     coredll:COREDLL.dll
 0003:000001b0       \177COREDLL_NULL_THUNK_DATA 000211b0     coredll:COREDLL.dll
 0003:000001b4       __imp_RIL_GetSystemTime    000211b4     ril:ril.dll
 0003:000001b8       __imp_RIL_GetSubscriberNumbers 000211b8     ril:ril.dll
 0003:000001bc       __imp_RIL_SendSupServiceData 000211bc     ril:ril.dll
 0003:000001c0       __imp_RIL_CancelSupServiceDataSession 000211c0     ril:ril.dll
 0003:000001c4       __imp_RIL_GetEquipmentState 000211c4     ril:ril.dll
 0003:000001c8       __imp_RIL_Initialize       000211c8     ril:ril.dll
 0003:000001cc       __imp_RIL_Deinitialize     000211cc     ril:ril.dll
 0003:000001d0       __imp_RIL_DevSpecific      000211d0     ril:ril.dll
 0003:000001d4       __imp_RIL_GetRegistrationStatus 000211d4     ril:ril.dll
 0003:000001d8       __imp_RIL_GetCallList      000211d8     ril:ril.dll
 0003:000001dc       \177ril_NULL_THUNK_DATA    000211dc     ril:ril.dll
 0003:000001e0       __imp_?GetAutoUpdateTimeUI@@YAKXZ 000211e0     sw_utilityG:sw_utilityG.dll
 0003:000001e4       __imp_?GetAutoUpdateTime@@YAKXZ 000211e4     sw_utilityG:sw_utilityG.dll
 0003:000001e8       __imp_?SetAutoUpdateTime@@YAXH@Z 000211e8     sw_utilityG:sw_utilityG.dll
 0003:000001ec       __imp_?GetRegValue@@YAJPAUHKEY__@@PBG1AAK@Z 000211ec     sw_utilityG:sw_utilityG.dll
 0003:000001f0       __imp_?GetCarrierIndex@@YAKXZ 000211f0     sw_utilityG:sw_utilityG.dll
 0003:000001f4       __imp_GetVersionInfo       000211f4     sw_utilityG:sw_utilityG.dll
 0003:000001f8       __imp_?SWAI_GetRegValue@@YAJPAUHKEY__@@PBG1PAEPAK@Z 000211f8     sw_utilityG:sw_utilityG.dll
 0003:000001fc       __imp_?GetRegValue@@YAJPAUHKEY__@@PBG1PAGPAK@Z 000211fc     sw_utilityG:sw_utilityG.dll
 0003:00000200       __imp_?SetRegValue@@YAJPAUHKEY__@@PBG11@Z 00021200     sw_utilityG:sw_utilityG.dll
 0003:00000204       __imp_?InWideMode@@YAHXZ   00021204     sw_utilityG:sw_utilityG.dll
 0003:00000208       __imp_?RelayoutDialog@@YAHPAUHINSTANCE__@@PAUHWND__@@PBG@Z 00021208     sw_utilityG:sw_utilityG.dll
 0003:0000020c       __imp_?GetActWizDisabled@@YAKXZ 0002120c     sw_utilityG:sw_utilityG.dll
 0003:00000210       __imp_?GetProductFeatures@@YAHAAK@Z 00021210     sw_utilityG:sw_utilityG.dll
 0003:00000214       __imp_?LogV@@YAXPBGZZ      00021214     sw_utilityG:sw_utilityG.dll
 0003:00000218       __imp_?GetVerInfo@@YAPAGPAUHINSTANCE__@@@Z 00021218     sw_utilityG:sw_utilityG.dll
 0003:0000021c       __imp_?InitLog@@YAXPAUHINSTANCE__@@@Z 0002121c     sw_utilityG:sw_utilityG.dll
 0003:00000220       __imp_?GetResolution@@YAHXZ 00021220     sw_utilityG:sw_utilityG.dll
 0003:00000224       __imp_?LogC@@YAXPBGZZ      00021224     sw_utilityG:sw_utilityG.dll
 0003:00000228       __imp_?LogStoreFileLine@@YAXPAGH@Z 00021228     sw_utilityG:sw_utilityG.dll
 0003:0000022c       __imp_?SWAI_GetRegValue@@YAJPAUHKEY__@@PBG1AAK@Z 0002122c     sw_utilityG:sw_utilityG.dll
 0003:00000230       \177sw_utilityG_NULL_THUNK_DATA 00021230     sw_utilityG:sw_utilityG.dll
 0003:00000234       __imp_Process32Next        00021234     toolhelp:toolhelp.dll
 0003:00000238       __imp_Process32First       00021238     toolhelp:toolhelp.dll
 0003:0000023c       __imp_CreateToolhelp32Snapshot 0002123c     toolhelp:toolhelp.dll
 0003:00000240       __imp_CloseToolhelp32Snapshot 00021240     toolhelp:toolhelp.dll
 0003:00000244       \177toolhelp_NULL_THUNK_DATA 00021244     toolhelp:toolhelp.dll
 0003:00000248       __xc_a                     00021248     corelibc:crt0init.obj
 0003:000003b4       __xc_z                     000213b4     corelibc:crt0init.obj
 0003:000003b8       __xi_a                     000213b8     corelibc:crt0init.obj
 0003:000003bc       __xi_z                     000213bc     corelibc:crt0init.obj
 0003:000003c0       __xp_a                     000213c0     corelibc:crt0init.obj
 0003:000003c4       __xp_z                     000213c4     corelibc:crt0init.obj
 0003:000003c8       __xt_a                     000213c8     corelibc:crt0init.obj
 0003:000003cc       __xt_z                     000213cc     corelibc:crt0init.obj
 0003:000003e0       ?TRAY_NOTIFYICON@@3IA      000213e0     MainFrm.obj
 0003:000003ec       ?szAppName@CSession@@2PAPBGA 000213ec     Session.obj
 0003:00000400       ??_R0?AVbad_alloc@std@@@8  00021400     SessionManager.obj
 0003:0000041c       ??_R0?AVexception@std@@@8  0002141c     SessionManager.obj
 0003:00000438       ??_R0?AVlength_error@std@@@8 00021438     SessionManager.obj
 0003:00000458       ??_R0?AVlogic_error@std@@@8 00021458     SessionManager.obj
 0003:00000484       ?m_SrvState@CModemStatus@@2KA 00021484     winmodemstat.obj
 0003:00000488       __security_cookie_complement 00021488     corelibc:seccook.obj
 0003:0000048c       __security_cookie          0002148c     corelibc:seccook.obj
 0003:00000494       ??_R0?AVout_of_range@std@@@8 00021494     libcpmt:string.obj
 0003:000004b8       _pRawDllMain               000214b8     atls:atlbase.obj
 0003:000004c0       ?hInst@@3PAUHINSTANCE__@@A 000214c0     AAM.obj
 0003:000004c4       ?theApp@@3VCAAMApp@@A      000214c4     AAM.obj
 0003:00000928       ?theMainWnd@@3VCMainFrame@@A 00021928     AAM.obj
 0003:00001450       ?m_MsgBoxBuffer@CModemStatus@@1UtagMsgBoxContent@@A 00022450     winmodemstat.obj
 0003:00001864       ?m_NonDataCallStatus@CModemStatus@@2KA 00022864     winmodemstat.obj
 0003:00001868       ?m_DataCallStatus@CModemStatus@@2KA 00022868     winmodemstat.obj
 0003:0000186c       ?m_CallType@CModemStatus@@2KA 0002286c     winmodemstat.obj
 0003:00001870       ?m_PwrState@CModemStatus@@2W4ePowerState@1@A 00022870     winmodemstat.obj
 0003:00001874       ?m_RoamState@CModemStatus@@2KA 00022874     winmodemstat.obj
 0003:00001878       ?m_IsOTASPCommited@CModemStatus@@2HA 00022878     winmodemstat.obj
 0003:0000187c       ?m_LastCallEndStatus@CModemStatus@@2GA 0002287c     winmodemstat.obj
 0003:00001880       ?m_hApi@CModemStatus@@1PAXA 00022880     winmodemstat.obj
 0003:00001884       ?m_hActiveWindow@CModemStatus@@2PAUHWND__@@A 00022884     winmodemstat.obj
 0003:00001888       ?m_MainWndH@CModemStatus@@1PAUHWND__@@A 00022888     winmodemstat.obj
 0003:0000188c       ?m_hCurrModPowerState@CModemStatus@@2PAXA 0002288c     winmodemstat.obj
 0003:00001890       ?m_hEquipmentStateOn@CModemStatus@@2PAXA 00022890     winmodemstat.obj
 0003:00001894       ?m_bDMMode@CModemStatus@@1HA 00022894     winmodemstat.obj
 0003:00001898       ?m_cFuncResultList@CModemStatus@@1V?$list@VCResultListElement@@V?$allocator@VCResultListElement@@@std@@@std@@A 00022898     winmodemstat.obj
 0003:000018a4       ?m_bInitFailed@CAtlBaseModule@ATL@@2_NA 000228a4     winmodemstat.obj
 0003:000018a8       ?_pAtlRawDllMain@@3P6AHPAXK0@ZA 000228a8     atls:atlbase.obj
 0003:000018ac       ?_AtlModuleInstance@ATL@@3PAUHINSTANCE__@@A 000228ac     atls:atlbase.obj
 0003:000018b0       ?_AtlBaseModule@ATL@@3VCAtlBaseModule@1@A 000228b0     atls:atlbase.obj
 0003:000018e4       __onexitend                000228e4     <common>
 0003:000018e8       __onexitbegin              000228e8     <common>
 0003:000018ec       _exitflag                  000228ec     <common>

 entry point at        0001:00008d70

 Static symbols

 0001:00000038       __unwind$59723             00011038 f i AAM.obj
 0001:00000108       __unwind$59791             00011108 f   AAM.obj
 0001:0000065c       __unwind$65126             0001165c f   Arbitrator.obj
 0001:0000066c       __unwind$65127             0001166c f   Arbitrator.obj
 0001:000013a4       __unwind$66459             000123a4 f   MainFrm.obj
 0001:000013c4       __unwind$66460             000123c4 f   MainFrm.obj
 0001:000013e4       __unwind$66461             000123e4 f   MainFrm.obj
 0001:00001400       __unwind$66462             00012400 f   MainFrm.obj
 0001:00001420       __unwind$66463             00012420 f   MainFrm.obj
 0001:00001440       __unwind$66464             00012440 f   MainFrm.obj
 0001:00001460       __unwind$66465             00012460 f   MainFrm.obj
 0001:0000147c       __unwind$66466             0001247c f   MainFrm.obj
 0001:0000149c       __unwind$66467             0001249c f   MainFrm.obj
 0001:000014bc       __unwind$66468             000124bc f   MainFrm.obj
 0001:000014dc       __unwind$66469             000124dc f   MainFrm.obj
 0001:000014f8       __unwind$66470             000124f8 f   MainFrm.obj
 0001:00001518       __unwind$66471             00012518 f   MainFrm.obj
 0001:00001538       __unwind$66472             00012538 f   MainFrm.obj
 0001:00001558       __unwind$66473             00012558 f   MainFrm.obj
 0001:00001574       __unwind$66474             00012574 f   MainFrm.obj
 0001:00001594       __unwind$66475             00012594 f   MainFrm.obj
 0001:000015b4       __unwind$66476             000125b4 f   MainFrm.obj
 0001:000016d8       __unwind$66586             000126d8 f   MainFrm.obj
 0001:000016f8       __unwind$66587             000126f8 f   MainFrm.obj
 0001:00001718       __unwind$66588             00012718 f   MainFrm.obj
 0001:00001734       __unwind$66589             00012734 f   MainFrm.obj
 0001:00001754       __unwind$66590             00012754 f   MainFrm.obj
 0001:00001774       __unwind$66591             00012774 f   MainFrm.obj
 0001:00001794       __unwind$66592             00012794 f   MainFrm.obj
 0001:000017b0       __unwind$66593             000127b0 f   MainFrm.obj
 0001:000017d0       __unwind$66594             000127d0 f   MainFrm.obj
 0001:000017f0       __unwind$66595             000127f0 f   MainFrm.obj
 0001:00001810       __unwind$66596             00012810 f   MainFrm.obj
 0001:0000182c       __unwind$66597             0001282c f   MainFrm.obj
 0001:0000184c       __unwind$66598             0001284c f   MainFrm.obj
 0001:0000186c       __unwind$66599             0001286c f   MainFrm.obj
 0001:0000188c       __unwind$66600             0001288c f   MainFrm.obj
 0001:000018a8       __unwind$66601             000128a8 f   MainFrm.obj
 0001:000018c8       __unwind$66602             000128c8 f   MainFrm.obj
 0001:000018e8       __unwind$66603             000128e8 f   MainFrm.obj
 0001:00004e58       __catch$61269              00015e58 f i SessionManager.obj
 0001:00004e84       __catch$61267              00015e84 f i SessionManager.obj
 0001:0000545c       __unwind$62041             0001645c f   SessionManager.obj
 0001:000056a8       __unwind$62667             000166a8 f i SessionManager.obj
 0001:000057f8       __unwind$62805             000167f8 f i SessionManager.obj
 0001:0000587c       __unwind$62894             0001687c f i SessionManager.obj
 0001:00005994       __unwind$63073             00016994 f   SessionManager.obj
 0001:00007728       __unwind$86855             00018728 f   winmodemstat.obj
 0001:000077d8       __unwind$87306             000187d8 f i winmodemstat.obj
 0001:00007938       __unwind$87556             00018938 f   winmodemstat.obj
 0001:00007950       __unwind$87557             00018950 f   winmodemstat.obj
 0001:000079dc       __catch$87638              000189dc f   winmodemstat.obj
 0001:00007bac       __catch$87712              00018bac f   winmodemstat.obj
 0001:00007ce0       __catch$87751              00018ce0 f   winmodemstat.obj
 0001:00008340       __catch$87871              00019340 f   winmodemstat.obj
 0001:00008558       __catch$87975              00019558 f   winmodemstat.obj
 0001:00008f74       doexit                     00019f74 f   corelibc:crt0dat.obj
 0001:000091b4       __unwind$17778             0001a1b4 f   libcpmt:string.obj
 0001:00009244       __unwind$17968             0001a244 f   libcpmt:string.obj
 0001:00009498       ?CanThisExceptionObjectBeDestructed@@YAEPAUEHExceptionRecord@@E@Z 0001a498 f   LIBCMT:frame_ce.obj
 0001:000097e4       ?CallCatchBlock@@YAPAXPAUEHExceptionRecord@@PAKPAU_CONTEXT@@PBU_s_FuncInfo@@PAXHK@Z 0001a7e4 f   LIBCMT:frame_ce.obj
 0001:00009b7c       ?BuildCatchObject@@YAXPAUEHExceptionRecord@@PAKPBU_s_HandlerType@@PBU_s_CatchableType@@@Z 0001ab7c f   LIBCMT:frame_ce.obj
 0001:00009d50       ?FindHandler@@YAEPAUEHExceptionRecord@@PAKPAU_CONTEXT@@PAU_DISPATCHER_CONTEXT@@PBU_s_FuncInfo@@H@Z 0001ad50 f   LIBCMT:frame_ce.obj
 0001:0000ab50       ??__EtheApp@@YAXXZ         0001bb50 f   AAM.obj
 0001:0000ab70       ??__EtheMainWnd@@YAXXZ     0001bb70 f   AAM.obj
 0001:0000ab90       ??__EIOTA_EXIT_MESSAGE@@YAXXZ 0001bb90 f   Arbitrator.obj
 0001:0000abb0       ??__EIOTA_BEGIN_MESSAGE@@YAXXZ 0001bbb0 f   MainFrm.obj
 0001:0000abd0       ??__EIOTA_END_MESSAGE@@YAXXZ 0001bbd0 f   MainFrm.obj
 0001:0000abf0       ??__EIOTA_BEGIN_ACK@@YAXXZ 0001bbf0 f   MainFrm.obj
 0001:0000ac10       ??__EIOTA_BEGIN_NACK@@YAXXZ 0001bc10 f   MainFrm.obj
 0001:0000ac30       ??__EIOTA_EXIT_MESSAGE@@YAXXZ 0001bc30 f   MainFrm.obj
 0001:0000ac50       ??__EIOTA_DIAL@@YAXXZ      0001bc50 f   MainFrm.obj
 0001:0000ac70       ??__EIOTA_1012_MIP_ERR@@YAXXZ 0001bc70 f   MainFrm.obj
 0001:0000ac90       ??__EPHONEUTILS_BEGIN_MESSAGE@@YAXXZ 0001bc90 f   MainFrm.obj
 0001:0000acb0       ??__EPHONEUTILS_END_MESSAGE@@YAXXZ 0001bcb0 f   MainFrm.obj
 0001:0000acd0       ??__EPHONEUTILS_BEGIN_ACK@@YAXXZ 0001bcd0 f   MainFrm.obj
 0001:0000acf0       ??__EPHONEUTILS_BEGIN_NACK@@YAXXZ 0001bcf0 f   MainFrm.obj
 0001:0000ad10       ??__EPHONEUTILS_EXIT_MESSAGE@@YAXXZ 0001bd10 f   MainFrm.obj
 0001:0000ad30       ??__EAW_BEGIN_MESSAGE@@YAXXZ 0001bd30 f   MainFrm.obj
 0001:0000ad50       ??__EAW_END_MESSAGE@@YAXXZ 0001bd50 f   MainFrm.obj
 0001:0000ad70       ??__EAW_BEGIN_ACK@@YAXXZ   0001bd70 f   MainFrm.obj
 0001:0000ad90       ??__EAW_BEGIN_NACK@@YAXXZ  0001bd90 f   MainFrm.obj
 0001:0000adb0       ??__EAW_EXIT_MESSAGE@@YAXXZ 0001bdb0 f   MainFrm.obj
 0001:0000add0       ??__EUPDATER_BEGIN@@YAXXZ  0001bdd0 f   MainFrm.obj
 0001:0000adf0       ??__EUPDATER_END@@YAXXZ    0001bdf0 f   MainFrm.obj
 0001:0000ae10       ??__EUPDATER_BEGIN_ACK@@YAXXZ 0001be10 f   MainFrm.obj
 0001:0000ae30       ??__EUPDATER_BEGIN_NACK@@YAXXZ 0001be30 f   MainFrm.obj
 0001:0000ae50       ??__EUPDATER_END_ACK@@YAXXZ 0001be50 f   MainFrm.obj
 0001:0000ae70       ??__EUPDATER_END_NACK@@YAXXZ 0001be70 f   MainFrm.obj
 0001:0000ae90       ??__EIOTA_BEGIN_NACK@@YAXXZ 0001be90 f   SessionManager.obj
 0001:0000aeb0       ??__EPHONEUTILS_EXIT_MESSAGE@@YAXXZ 0001beb0 f   SessionManager.obj
 0001:0000aed0       ??__EPOWER_ON@@YAXXZ       0001bed0 f   StdAfx.obj
 0001:0000aef0       ??__EPOWER_OFF@@YAXXZ      0001bef0 f   StdAfx.obj
 0001:0000af10       ??__EIOTA_BEGIN_MESSAGE@@YAXXZ 0001bf10 f   StdAfx.obj
 0001:0000af30       ??__EIOTA_END_MESSAGE@@YAXXZ 0001bf30 f   StdAfx.obj
 0001:0000af50       ??__EIOTA_BEGIN_ACK@@YAXXZ 0001bf50 f   StdAfx.obj
 0001:0000af70       ??__EIOTA_BEGIN_NACK@@YAXXZ 0001bf70 f   StdAfx.obj
 0001:0000af90       ??__EIOTA_END_ACK@@YAXXZ   0001bf90 f   StdAfx.obj
 0001:0000afb0       ??__EIOTA_EXIT_MESSAGE@@YAXXZ 0001bfb0 f   StdAfx.obj
 0001:0000afd0       ??__EIOTA_ALIVE_MESSAGE@@YAXXZ 0001bfd0 f   StdAfx.obj
 0001:0000aff0       ??__EIOTA_PING_MESSAGE@@YAXXZ 0001bff0 f   StdAfx.obj
 0001:0000b010       ??__EIOTA_PING_ACK@@YAXXZ  0001c010 f   StdAfx.obj
 0001:0000b030       ??__EIOTA_CRITICAL_ERROR@@YAXXZ 0001c030 f   StdAfx.obj
 0001:0000b050       ??__EIOTA_NON_CRITICAL_ERROR@@YAXXZ 0001c050 f   StdAfx.obj
 0001:0000b070       ??__EIOTA_KILL_ME@@YAXXZ   0001c070 f   StdAfx.obj
 0001:0000b090       ??__EIOTA_UPDATE_STATUS@@YAXXZ 0001c090 f   StdAfx.obj
 0001:0000b0b0       ??__EIOTA_DATAPORT_INUSE@@YAXXZ 0001c0b0 f   StdAfx.obj
 0001:0000b0d0       ??__EIOTA_DONE@@YAXXZ      0001c0d0 f   StdAfx.obj
 0001:0000b0f0       ??__EIOTA_DIAL@@YAXXZ      0001c0f0 f   StdAfx.obj
 0001:0000b110       ??__EIOTA_1012_MIP_ERR@@YAXXZ 0001c110 f   StdAfx.obj
 0001:0000b130       ??__EPHONEUTILS_BEGIN_MESSAGE@@YAXXZ 0001c130 f   StdAfx.obj
 0001:0000b150       ??__EPHONEUTILS_END_MESSAGE@@YAXXZ 0001c150 f   StdAfx.obj
 0001:0000b170       ??__EPHONEUTILS_BEGIN_ACK@@YAXXZ 0001c170 f   StdAfx.obj
 0001:0000b190       ??__EPHONEUTILS_BEGIN_NACK@@YAXXZ 0001c190 f   StdAfx.obj
 0001:0000b1b0       ??__EPHONEUTILS_END_ACK@@YAXXZ 0001c1b0 f   StdAfx.obj
 0001:0000b1d0       ??__EPHONEUTILS_EXIT_MESSAGE@@YAXXZ 0001c1d0 f   StdAfx.obj
 0001:0000b1f0       ??__EPHONEUTILS_ALIVE_MESSAGE@@YAXXZ 0001c1f0 f   StdAfx.obj
 0001:0000b210       ??__EPHONEUTILS_PING_MESSAGE@@YAXXZ 0001c210 f   StdAfx.obj
 0001:0000b230       ??__EPHONEUTILS_PING_ACK@@YAXXZ 0001c230 f   StdAfx.obj
 0001:0000b250       ??__EAW_BEGIN_MESSAGE@@YAXXZ 0001c250 f   StdAfx.obj
 0001:0000b270       ??__EAW_END_MESSAGE@@YAXXZ 0001c270 f   StdAfx.obj
 0001:0000b290       ??__EAW_BEGIN_ACK@@YAXXZ   0001c290 f   StdAfx.obj
 0001:0000b2b0       ??__EAW_BEGIN_NACK@@YAXXZ  0001c2b0 f   StdAfx.obj
 0001:0000b2d0       ??__EAW_END_ACK@@YAXXZ     0001c2d0 f   StdAfx.obj
 0001:0000b2f0       ??__EAW_EXIT_MESSAGE@@YAXXZ 0001c2f0 f   StdAfx.obj
 0001:0000b310       ??__EAW_ALIVE_MESSAGE@@YAXXZ 0001c310 f   StdAfx.obj
 0001:0000b330       ??__EAW_PING_MESSAGE@@YAXXZ 0001c330 f   StdAfx.obj
 0001:0000b350       ??__EAW_PING_ACK@@YAXXZ    0001c350 f   StdAfx.obj
 0001:0000b370       ??__EUPDATER_BEGIN@@YAXXZ  0001c370 f   StdAfx.obj
 0001:0000b390       ??__EUPDATER_END@@YAXXZ    0001c390 f   StdAfx.obj
 0001:0000b3b0       ??__EUPDATER_BEGIN_ACK@@YAXXZ 0001c3b0 f   StdAfx.obj
 0001:0000b3d0       ??__EUPDATER_BEGIN_NACK@@YAXXZ 0001c3d0 f   StdAfx.obj
 0001:0000b3f0       ??__EUPDATER_END_ACK@@YAXXZ 0001c3f0 f   StdAfx.obj
 0001:0000b410       ??__EUPDATER_END_NACK@@YAXXZ 0001c410 f   StdAfx.obj
 0001:0000b430       ??__ERIL_STATUS_CHANGED@@YAXXZ 0001c430 f   StdAfx.obj
 0001:0000b450       ??__ERIL_DBG_NOTIFY@@YAXXZ 0001c450 f   StdAfx.obj
 0001:0000b470       ??__ERIL_TECHHDR_NOTIFY@@YAXXZ 0001c470 f   StdAfx.obj
 0001:0000b490       ??__ERIL_IOTA_STATUS_CHANGED@@YAXXZ 0001c490 f   StdAfx.obj
 0001:0000b4b0       ??__ERIL_IOTA_WAP_URI@@YAXXZ 0001c4b0 f   StdAfx.obj
 0001:0000b4d0       ??__ERIL_PDSM_PD_DATA@@YAXXZ 0001c4d0 f   StdAfx.obj
 0001:0000b4f0       ??__ERIL_PDSM_PD_DONE@@YAXXZ 0001c4f0 f   StdAfx.obj
 0001:0000b510       ??__ERIL_PDSM_PD_END@@YAXXZ 0001c510 f   StdAfx.obj
 0001:0000b530       ??__ERIL_PDSM_PD_BEGIN@@YAXXZ 0001c530 f   StdAfx.obj
 0001:0000b550       ??__ERIL_PDSM_PD_UPDATE_FAILURE@@YAXXZ 0001c550 f   StdAfx.obj
 0001:0000b570       ??__ERIL_PDSM_PD_DLD_DATA@@YAXXZ 0001c570 f   StdAfx.obj
 0001:0000b590       ??__ERIL_PDSM_PD_DLD_DONE@@YAXXZ 0001c590 f   StdAfx.obj
 0001:0000b5b0       ??__ERIL_PDSM_PD_DLD_END@@YAXXZ 0001c5b0 f   StdAfx.obj
 0001:0000b5d0       ??__ERIL_PDSM_PD_DLD_BEGIN@@YAXXZ 0001c5d0 f   StdAfx.obj
 0001:0000b5f0       ??__ERIL_PDSM_PA_PARAM@@YAXXZ 0001c5f0 f   StdAfx.obj
 0001:0000b610       ??__ERIL_CALL_BYTE_CTR@@YAXXZ 0001c610 f   StdAfx.obj
 0001:0000b630       ??__E?m_cFuncResultList@CModemStatus@@1V?$list@VCResultListElement@@V?$allocator@VCResultListElement@@@std@@@std@@A@@YAXXZ 0001c630 f   winmodemstat.obj
 0001:0000b664       ??__E_AtlBaseModule@ATL@@YAXXZ 0001c664 f   atls:atlbase.obj
 0001:0000b6a0       ??__FtheMainWnd@@YAXXZ     0001c6a0 f   AAM.obj
 0001:0000b6ac       ??__FtheApp@@YAXXZ         0001c6ac f   AAM.obj
 0001:0000b6b8       ??__F?m_cFuncResultList@CModemStatus@@1V?$list@VCResultListElement@@V?$allocator@VCResultListElement@@@std@@@std@@A@@YAXXZ 0001c6b8 f   winmodemstat.obj
 0001:0000b6e0       ??__F_AtlBaseModule@ATL@@YAXXZ 0001c6e0 f   atls:atlbase.obj
